:100000002BC3000048C3000046C3000044C30000E7
:1000100042C3000040C300003EC300003CC30000D8
:100020003AC3000038C3000036C3000034C30000E8
:100030000C94383830C300002EC300002CC30000DD
:100040002AC3000028C300000C94243824C30000F5
:1000500022C3000020C300001EC300001CC3000018
:100060001AC3000018C3000016C3000014C3000028
:1000700012C3000010C300000EC300000CC3000038
:100080000AC3000008C3000006C300003D0984093C
:10009000B409E4093C0A570A870AB70A200BE70AA1
:1000A00062096709D70ADC0AE10A75097A097F093A
:1000B000580D640D670D6A0D6D0D7B0DBF0DBF0DE5
:1000C000960DA30DA710AC10BA10BF10C410C91024
:1000D000CE10D310551558155B155E1561156415B6
:1000E00067156A15E21E071F1B1F2E1F311F421FB7
:1000F000531F711FF81EFB1E641F671F6A1FFE1E21
:10010000011F041F6E24732478247D2482248724F5
:100110008C24912497249A244E26B926DD2746283C
:100120006529912A772B6C2C9B2DEA2D4D2E972E2D
:100130009E2EF22E472F4A2F4D2F502F532F562FE2
:10014000592F5C2FF8310E3224323B325132673254
:100150007D329332E732EA32ED32F032F332F63268
:10016000F932FC3236334B33603373338633943396
:10017000A733BA33CD33E233F7330C342B34443462
:10018000000000000000000004040404000400005B
:100190000A0A0A00000000000A0A1F0A1F0A0A00D1
:1001A000040F140E051E040018190204081303009E
:1001B0000C12140814120D000C04080000000000BA
:1001C00002040808080402000804020202040800ED
:1001D0000004150E150400000004041F04040000B0
:1001E000000000000C0408000000001F00000000D8
:1001F00000000000000C0C000001020408100000C8
:100200000E11131519110E00040C040404040E0041
:100210000E11010204081F001F02040201110E004A
:1002200002060A121F0202001F101E0101110E0019
:100230000608101E11110E001F0102040808080014
:100240000E11110E11110E000E11110F01020C00F2
:100250000001020408100000000C0C000C0408004F
:10026000020408100804020000001F001F00000024
:1002700008040201020408000E1101020400040037
:100280000E11010D15150E000E1111111F11110087
:100290001E11111E11111E000E11101010110E0052
:1002A0001C12111111121C001F10101E10101F0023
:1002B0001F10101E101010000E11101711110E003B
:1002C0001111111F111111000E04040404040E0079
:1002D0000702020202120C0011121418141211006B
:1002E0001010101010101F00111B15151111110006
:1002F00011111915131111000E11111111110E0008
:100300001E11111E101010000E11111115120D00EA
:100310001E11111E141211000F10100E01011E00EB
:100320001F040404040404001111111111110E0022
:1003300011111111110A04001111111115150E00DE
:1003400011110A040A1111001111110A0404040008
:100350001F01020408101F000E08080808080E00FC
:10036000110A1F041F0404000E02020202020E0002
:10037000040A1100000000000000000000001F003F
:10038000080400000000000000000E010F110F0023
:1003900010101E1111111E0000000E1010110E0081
:1003A00001010D1311110F0000000E111F100E009E
:1003B0000609081C08080800000F11110F010E00A3
:1003C000101016191111110004000C0404040E0081
:1003D0000200060202120C0010101214181412006F
:1003E0001808080808081C0000001A15151111004B
:1003F000000016191111110000000E1111110E004C
:1004000000001E111E10100000000F110F0101004E
:10041000000016191010100000000E100E011E0032
:1004200008081C08080906000000111111130D002E
:1004300000001111110A04000000111111150A0029
:100440000000110A040A1100000011110F010E0032
:1004500000001F0204081F00384444447C44440048
:100460007C404078444478007844447844447800A0
:100470007C404040404040000C14242424243C4450
:100480007C40407840407C005454543854545400CC
:10049000384404180444380044444C546444440030
:1004A00054444C5464444400444850605048440010
:1004B0001C24242424246400446C545444444400E4
:1004C0004444447C44444400384444444444380054
:1004D0007C444444444444007844447840404000D0
:1004E00038444040404438007C1010101010100078
:1004F0004444443C044438003854545438101000E8
:1005000044442810284444004444444444447E0263
:10051000444444443C0404005454545454547C0013
:100520005454545454547E026020203824243800FB
:100530004444446454546400404040784444780047
:100540003844041C0444380048545474545448003B
:100550003C44443C14244400000038043C443C0027
:1005600000007840784478000000784C784C78009F
:1005700000007840404040000000182828287C44B3
:10058000000038447C403C0000005454385454006F
:1005900000007804380478000000444C546444009F
:1005A0000010444C54644400000044487048440027
:1005B00000001C24444444000000446C5454440093
:1005C0000000484878484800000038444444380057
:1005D00000007848484848000000704870404000DB
:1005E000000038404040380000007C10101010001F
:1005F0000000484838087000000038545438100093
:1006000000004428102844000000484848487C0462
:1006100000004848380808000000545454547C0036
:100620000000545454547E02000060203C223C00E0
:1006300000004242724A7200000040407844780054
:10064000000070087808700000004C5272524C0094
:1006500000003C443C44440011241FBECFEFD0E1D5
:10066000DEBFCDBF16E0A0E0B1E0E4E1FEE800E0CF
:100670000BBF02C007900D92AC31B107D9F726E04D
:10068000ACE1B6E001C01D92AA3DB207E1F70E94BD
:1006900096380C940847B4CCE2E6F0E090819E7F57
:1006A00090839081946090839081977F9083A898A5
:1006B0008BBB8DE08A95F1F70000A89A8081886055
:1006C00080830895E2E6F0E09081916090839081CC
:1006D000946090839081977F9083A8988BBB8DE0E6
:1006E0008A95F1F70000A89A808188608083089538
:1006F000CF93C82F892FE6DF8C2FCF91E3CFE2E68F
:10070000F0E02081216020832081246020832081EB
:10071000277F2083A8988BBB92BB8DE08A95F1F749
:100720000000A89A8081886080830895CF93C82FA5
:1007300086E3B2DFC13049F030F0C23041F0C3305F
:1007400059F488EE07C088E403C088E203C088E853
:10075000B9DF04C0B7DF0BC0CD7F49F48FEE90E066
:1007600090931F0680931E068FE391E008C08FE3ED
:1007700091E090931F0680931E068FEE90E0909379
:100780001D0680931C06CF910895CF93C82F8FEF3D
:100790008ABB81BB8093610081E084BBE2E6F0E02C
:1007A00080818260808381E077DF2FEF89E698E1A6
:1007B000215080409040E1F700C0000080EC6CDFE9
:1007C00085E280DF81EC68DF81E17CDF85EC64DF3E
:1007D0008BE278DF8BE276DF87EC5EDF86E872DF24
:1007E0008C2FA4DF8AE358DF85E06CDF81EB54DFD8
:1007F00080E068DF88E166DF86EB4EDF8AE062DF5B
:1008000082E860DF87E25EDF81E146DF2FEF8DEE79
:1008100092E0215080409040E1F700C0000089E262
:10082000CF913ACF0F931F93CF93DF938C01EB01BE
:100830008AE232DFC8015CDFCE01DF91CF911F91E8
:100840000F9156CF0F931F93CF93DF938C01EB0142
:100850008BE222DFC8014CDFCE01DF91CF911F91E7
:100860000F9146CFCF93DF93EB01BC01DBDFBE01DD
:10087000CE01E8DF8CE2DF91CF910ECFCF93DF93F3
:10088000EA01F0DFCE01DF91CF9139CF8F929F92B5
:10089000AF92BF92CF92DF92EF92FF920F931F938E
:1008A000CF93DF93A8956817790738F486279727A1
:1008B0006827792786279727A8952417350738F4BE
:1008C000422753272427352742275327A895A0914D
:1008D0001E06B0911F06FC01A817B90708F4FD0118
:1008E0006B01A617B70708F46D0180911C06909163
:1008F0001D06EA018417950708F4EC0179018217B7
:10090000930708F47C01A89596012F5F3F4F2E1B9B
:100910003F0BD7011196AC1BBD0B0E94D0434B017E
:100920005C01B601CF017EDFA895B701CE018ADF59
:100930008CE2B2DEA895C12CD12C7601C814D90462
:10094000EA04FB0449F0C801DADEA8958FEFC81A63
:10095000D80AE80AF80AF2CFDF91CF911F910F91E0
:10096000FF90EF90DF90CF90BF90AF909F908F90CF
:1009700008950F931F934115510579F02115310505
:1009800061F0FA01AB0161507109260F371FBC01FC
:10099000615071096E0F7F1F79DF1F910F910895CC
:1009A0002F923F924F925F926F927F928F929F927F
:1009B000AF92BF92CF92DF92EF92FF920F931F936D
:1009C000CF93DF93CDB7DEB767970FB6F894DEBF4E
:1009D0000FBECDBF5C01798B688B598748873B87F9
:1009E0002A870F83F12C28E0029FC00111241A826C
:1009F0001982E8E0F0E0FF8BEE8B47019C01285F55
:100A000031093B8B2A8BFC01E052F340FD8BEC8BD0
:100A1000C888D98889819A81C80ED91E8A899B89FC
:100A2000EE89FF898E1B9F0B9C0120583E4F3F870C
:100A30002E878C899D898E1B9F0BFC01E058FE4FF1
:100A4000FD87EC871E821D821C821B8287E0682E38
:100A5000712C412C512C212C312CFF81F7FD1EC013
:100A6000EE85FF85849190E0062C02C095958795D0
:100A70000A94E2F780FF08C0088519859701A7014D
:100A8000B6018D819E8107C00A851B859701A7014C
:100A9000B6018B819C818A0D9B1D20C0FF81F03C9B
:100AA000F0F0EC85FD85849190E0062C02C09595D0
:100AB00087950A94E2F780FF09C008851985970198
:100AC000A701B601C501820D931D08C00A851B85CB
:100AD0009701A701B601C501840D951D4ADF280CB9
:100AE000391C480C591CF1E06F1A71082B813C81AC
:100AF000280D391D3C832B838D819E81880D991D86
:100B00009E838D839FEF6916790609F0A6CFEE8943
:100B1000FF893197FF8BEE8B29813A812E0D3F1D86
:100B20003A832983EF2B09F073CF67960FB6F894B9
:100B3000DEBF0FBECDBFDF91CF911F910F91FF9010
:100B4000EF90DF90CF90BF90AF909F908F907F906D
:100B50006F905F904F903F902F9008954F925F92CB
:100B60006F927F928F929F92AF92BF92CF92DF92BD
:100B7000EF92FF920F931F93CF93DF93EC016B01E2
:100B80004A013901102F88E0089F500111242701E4
:100B9000F20101912F010023B1F020911E06309146
:100BA0001F06CE0108962817390720F4CA0CDB1C53
:100BB000C1E0D0E0E12E9301A401B601CE01F0DE48
:100BC000CA0DDB1DE5CFDF91CF911F910F91FF90F3
:100BD000EF90DF90CF90BF90AF909F908F907F90DD
:100BE0006F905F904F9008956F927F928F929F9237
:100BF000AF92BF92CF92DF92EF92FF920F93CF937B
:100C0000DF9300D000D0CDB7DEB76C015B014A01A5
:100C10003901C70119821A821B821C824AE0BE0177
:100C20006F5F7F4F0E94DF43CE0101967C019301ED
:100C3000A401B501C60192DF0F900F900F900F90A5
:100C4000DF91CF910F91FF90EF90DF90CF90BF9009
:100C5000AF909F908F907F906F9008950F931F9308
:100C600020911C0630911D0660911E0670911F0692
:100C70008C0140E050E080E090E008DE1F910F9191
:100C800008956F927F928F929F92AF92BF92CF9270
:100C9000DF92EF92FF920F93CF93DF936C01EB0102
:100CA0007A0159014C01840E951EB401BBDDBE01D1
:100CB000CE01C8DD8CE2F0DC612C712C6E147F0457
:100CC00031F0C5011CDD8FEF681A780AF7CF0230CA
:100CD00008F43EC0B401C601A5DDCE010196BC01F9
:100CE000B1DD8CE2D9DC612C712C6E147F0431F003
:100CF000C50105DD8FEF681A780AF7CF023041F1A0
:100D0000B401C6018FDDCE010296BC019BDD8CE2F1
:100D1000C3DC612C712C6E147F0431F0C501EFDC53
:100D20008FEF681A780AF7CF033091F0B401C6014B
:100D300079DDCE010396BC0185DD8CE2ADDCC0E03F
:100D4000D0E0CE15DF0521F0C501D9DC2196F9CF21
:100D5000DF91CF910F91FF90EF90DF90CF90BF90F8
:100D6000AF909F908F907F906F9008956F927F9239
:100D70008F929F92AF92BF92CF92DF92EF92FF92AB
:100D80000F93CF93DF93EC016B017A015901BC0102
:100D900049DD46018E0C9F1CB401C60153DD8CE277
:100DA0007BDC612C712C6E147F0431F0C501A7DC53
:100DB0008FEF681A780AF7CF023008F43EC0CE01F0
:100DC0000196BC012FDDB401C6013CDD8CE264DC80
:100DD000612C712C6E147F0431F0C50190DC8FEF13
:100DE000681A780AF7CF023041F1CE010296BC01B1
:100DF00019DDB401C60126DD8CE24EDC612C712CBC
:100E00006E147F0431F0C5017ADC8FEF681A780A1E
:100E1000F7CF033091F0CE010396BC0103DDB4019E
:100E2000C60110DD8CE238DCC0E0D0E0CE15DF0575
:100E300021F0C50164DC2196F9CFDF91CF910F91AC
:100E4000FF90EF90DF90CF90BF90AF909F908F90EA
:100E50007F906F9008956F927F928F929F92AF9242
:100E6000BF92CF92DF92EF920F931F93CF93DF93B6
:100E70006C015B01EA01390148010E2D940101DF8B
:100E8000B301615071096A0D7B1D9401AE01C60169
:100E9000F8DE9401A301B501C60168DFCE01019718
:100EA0009401A301B5018C0D9D1D60DFDF91CF91F1
:100EB0001F910F91EF90DF90CF90BF90AF909F90D8
:100EC0008F907F906F900895EF92FF920F931F93F2
:100ED000CF93DF93EB018A017901BC01640F751F89
:100EE000A1DCBE01CE01AEDC8CE2D6DBC0E0D0E0FE
:100EF000C017D10721F0C70102DC2196F9CFDF919D
:100F0000CF911F910F91FF90EF900895EF92FF9274
:100F10000F931F93CF93DF93EB018A017901BC01FB
:100F200081DCBE01600F711FCE018CDC8CE2B4DB72
:100F3000C0E0D0E0C017D10721F0C701E0DB219667
:100F4000F9CFDF91CF911F910F91FF90EF9008950E
:100F50002F923F924F925F926F927F928F929F92C9
:100F6000AF92BF92CF92DF92EF92FF920F931F93B7
:100F7000CF93DF9300D000D000D0CDB7DEB76C01A7
:100F80007B015A0139012801261B370B3A8329833B
:100F90008A01081B190B17FF03C011950195110950
:100FA000CA14DB0420F022242A94322C03C0222409
:100FB0002394312C89819A819E838D8397FF05C06C
:100FC0009195819591099E838D832D813E813195E7
:100FD000219531093C832B83E614F70428F08FEF29
:100FE0009FEF9A83898304C021E030E03A8329830C
:100FF00048018D819E81881A990AA201B701C60114
:101000003DDCC401880F991F2B813C818217930717
:1010100064F0CA14DB0499F02D813E81821A930A90
:10102000C20CD31C0817190744F3E614F70439F06F
:10103000800E911E89819A81E80EF91EDECF2696D8
:101040000FB6F894DEBF0FBECDBFDF91CF911F91D9
:101050000F91FF90EF90DF90CF90BF90AF909F9057
:101060008F907F906F905F904F903F902F9008955A
:10107000AF92BF92CF92DF92EF92FF920F931F93A6
:10108000CF93DF937C016B01EA01590198011CDFCA
:10109000B501615071096C0D7D1D9801AE01C7014C
:1010A00013DF9801A501B601C70130DFCE0101971A
:1010B0009801A501B6018E0D9F1DDF91CF911F9163
:1010C0000F91FF90EF90DF90CF90BF90AF901ECF29
:1010D0002F923F924F925F926F927F928F929F9248
:1010E000AF92BF92CF92DF92EF92FF920F931F9336
:1010F000CF93DF931C012B01690150E000271127DA
:10110000041B150BC1E0D0E0C41BD50BCC0FDD1FB9
:10111000E12CF12CA6015701A40CB51CB50131013D
:10112000601A710AC301AADBA601B5014801820C4D
:10113000931CC401A3DBA6015201AE18BF08B50180
:10114000C4019CDBA601B501C30198DBEC16FD06CA
:10115000B4F08FEFE81AF80AC701880F991F0196BB
:101160008C0F9D1F22273327201B310BE216F3061D
:1011700039F40C171D074CF0C0E0D0E001C0CE01DF
:101180000C171D0714F0EC01C5CF0F5F1F4F98011E
:10119000220F331F2F5F3F4F820F931F1016110630
:1011A00094F7DF91CF911F910F91FF90EF90DF9017
:1011B000CF90BF90AF909F908F907F906F905F90F7
:1011C0004F903F902F9008954F925F926F927F9231
:1011D0008F929F92AF92BF92CF92DF92EF92FF9247
:1011E0000F931F93CF93DF93EC015B014A01390109
:1011F00028018601ADDE9701A201B301C401A8DE7A
:101200009501AE01B701C201A3DEDF91CF911F911D
:101210000F91FF90EF90DF90CF90BF90AF909F9095
:101220008F907F906F905F904F900895CF93C82FCD
:101230008A3011F48DE0FADF5D9BFECFCCB980E0FF
:1012400090E0CF910895CF92DF92EF92FF920F93AB
:101250001F93CF93DF93CDB7DEB761970FB6F894A6
:10126000DEBF0FBECDBF90E08A30910508F0E8C127
:10127000FC01EA5BFF4F0C94C743A8958AE0E4E3C6
:10128000F1E0DE01119601900D928A95E1F7CE0111
:1012900001967C0101E02FE130E04FEF5FEF63E268
:1012A00070E08AE090E05ADCA895E091C0068E2FAD
:1012B00090E08830910508F0C3C1FC01E05BFF4F6E
:1012C0000C94C743A4E8EA2EA5E0FA2E04C0FFE779
:1012D000EF2EF5E0FF2E02E02FE130E04FEF5FEF61
:1012E0006EE170E08BEE90E0AAC1E7E5EE2EE5E05E
:1012F000FE2E6BC17DE4E72E75E0F72E66C163E438
:10130000E62E65E0F62E61C1A89588E0EEE3F1E0F7
:10131000DE01119601900D928A95E1F786E0E3EAED
:10132000F1E0DE011C9601900D928A95E1F7CE0165
:1013300001967C0101E02FE130E04FEF5FEF64E1C7
:1013400070E084E190E00ADCCE010C967C012FE194
:1013500030E04FEF5FEF68E270E08EE190E0FEDB9F
:10136000A89580916E061DC1A89587E0E6E4F1E09E
:10137000DE01119601900D928A95E1F786E0E3EA8D
:10138000F1E0DE011C9601900D928A95E1F7CE0105
:1013900001967C0101E02FE130E04FEF5FEF64E167
:1013A00070E084E190E0DADBCE010C967C012FE165
:1013B00030E04FEF5FEF68E270E08EE190E0CEDB6F
:1013C000A89580917506EDC0A89587E0EDE4F1E061
:1013D000DE01119601900D928A95E1F7CE010196FA
:1013E0007C0101E02FE130E04FEF5FEF63E270E05E
:1013F00089E190E0B3DBA8952FE130E04FEF5FEF9C
:101400006EE170E08EEE90E0A9DB30EEC32E37E0A7
:10141000D32E41E6E42EF12C0EE110E021E630E07F
:101420004AE050E067E570E084E190E0CDDE06E35D
:1014300011E021E630E042E251E067E570E08CE245
:1014400091E0C2DE50EAE52EF12C0EE110E020EA38
:1014500030E04AE050E06AEA70E084E190E0B4DE17
:1014600006E311E020EA30E042E251E06AEA70E08F
:101470008CE291E0A9DEE4C0A8958BE0E4E5F1E020
:10148000DE01119601900D928A95E1F7CE01019649
:101490007C0101E02FE130E04FEF5FEF63E270E0AD
:1014A0008FE090E05BDBA8958091CA067AC0A89592
:1014B00086E0EFE5F1E0DE011C9601900D928A9541
:1014C000E1F78AE0E5E6F1E0DE01119601900D9288
:1014D0008A95E1F7CE010C967C0101E02FE130E026
:1014E0004FEF5FEF64E170E089E190E037DBCE0120
:1014F00001967C012FE130E04FEF5FEF63E270E097
:101500008FE090E02BDBA8958091BF064AC0A8959C
:1015100086E0EFE5F1E0DE01119601900D928A95EB
:10152000E1F785E0EFE6F1E0DE011C9601900D9217
:101530008A95E1F7CE0101967C0101E02FE130E0D0
:101540004FEF5FEF64E170E089E190E007DBCE01EF
:101550000C967C012FE130E04FEF5FEF63E270E02B
:101560008FE190E0FBDAA8958091BC061AC0A8959F
:1015700088E0E4E7F1E0DE01119601900D928A9592
:10158000E1F7CE0101967C0101E02FE130E04FEF61
:101590005FEF63E270E08FE090E0E0DAA895809181
:1015A0007C06813049F018F0823059F049C025E7B7
:1015B000E22E25E0F22E09C09BE6E92E95E0F92EF9
:1015C00004C081E6E82E85E0F82E01E030C0A89541
:1015D0008BE0ECE7F1E0DE01119601900D928A9527
:1015E000E1F785E0E7E8F1E0DE011C9601900D925D
:1015F0008A95E1F7CE0101967C0101E02FE130E010
:101600004FEF5FEF64E170E08AE090E0A7DACE018F
:101610000C967C012FE130E04FEF5FEF68E270E065
:101620008EE190E09BDAA895CE0101967C012FE136
:1016300030E04FEF5FEF6EE170E086EE90E08EDA23
:1016400061960FB6F894DEBF0FBECDBFDF91CF918C
:101650001F910F91FF90EF90DF90CF900895CF935F
:10166000DF9300D000D0CDB7DEB78091630080FD5E
:1016700021C01C821B821A821982BE016F5F7F4FBC
:10168000CE0103960E9426428B819C81853C994025
:1016900088F0A89589819A81843C994058F4A8954E
:1016A00089819A818D3D954028F0A89581E08093AD
:1016B0006706A8950F900F900F900F90DF91CF9134
:1016C0000895CF93DF9300D000D0CDB7DEB7A895B3
:1016D0008091630080FD23C01C821B821A821982C4
:1016E000BE016F5F7F4FCE0103960E9426428B8121
:1016F0009C81853C994098F089819A81843C9940ED
:1017000070F489819A818D3D954048F0109267066A
:101710008FE19EE40197F1F700C00000A8950F90BB
:101720000F900F900F90DF91CF910895CF92DF929D
:10173000EF92FF920F931F93A895809167068111F6
:1017400040C0A8950FE110E02CE430E04EE650E0F8
:101750006CE870E089E690E00CD920E038EF48E2D0
:1017600064EB70E080EA90E0B3DC20E038EF47E221
:1017700064EB70E080EA90E0ABDC20E038EF4BE215
:1017800064EB70E080EA90E0A3DC20E038EF45E213
:1017900064EB70E080EA90E09BDC00E018EF23E26D
:1017A00030E045E050E065EA70E086E990E0E1D89D
:1017B00023E230E045E050E065EA70E085EA90E041
:1017C000D8D880916706813009F03EC0A8950FE116
:1017D00010E02CE430E04EE650E06CE870E089E682
:1017E00090E0C7D820EE37E048E264EB70E080EA92
:1017F00090E06EDC20EE37E047E264EB70E080EAD8
:1018000090E066DC20EE37E04BE264EB70E080EACB
:1018100090E05EDC20EE37E045E264EB70E080EAC9
:1018200090E056DC80EEC82E87E0D82E94EBE92EAF
:10183000F12C07EB10E028EC30E044E950E060EADE
:1018400070E084E990E0C0DC1F910F91FF90EF9071
:10185000DF90CF900895EF92FF920F931F93CF9355
:10186000DF93CDB7DEB764970FB6F894DEBF0FBE37
:10187000CDBFA8950FEF1FEF21E430E04FE550E01A
:1018800065E070E085E090E0F3DBA89521E430E0CE
:101890004FE550E06BE470E085E090E0E9DB2BE49D
:1018A00030E04FE550E061E970E085E090E0E0DB9A
:1018B00089E0ECE8F1E0DE01119601900D928A9545
:1018C000E1F785E0E7E8F1E0DE01509601900D9246
:1018D0008A95E1F7CE0101967C0101E02FE130E02D
:1018E0004FEF5FEF60E570E082E190E037D9CE0125
:1018F00040967C012FE130E04FEF5FEF6AE570E04A
:1019000083E290E02BD90FEF1FEF21E430E04FE5A9
:1019100050E065E070E08CED90E0AADB21E430E07F
:101920004FE550E06BE470E08CED90E0A1DB2BE440
:1019300030E04FE550E061E970E08CED90E098DB3D
:1019400086E0E5E9F1E0DE011A9601900D928A95B4
:10195000E1F7CE0101967C0101E02FE130E04FEF8D
:101960005FEF60E570E08BEE90E0F8D8CE010A966C
:101970007C012FE130E04FEF5FEF6AE570E08CEF24
:1019800090E0ECD885E3E82E83E0F82E2FE130E0FC
:101990004FEF5FEF66EE70E08AE090E0DFD8C6DEE2
:1019A0008091680650DC64960FB6F894DEBF0FBED7
:1019B000CDBFDF91CF911F910F91FF90EF900895D0
:1019C000EF92FF920F93CF93DF93CDB7DEB7CE5652
:1019D000D1090FB6F894DEBF0FBECDBF9AE0E4E3A5
:1019E000F1E0DE01A75ABF4F01900D929A95E1F701
:1019F0009EE0EBE9F1E0DE015E9601900D929A9592
:101A0000E1F79EE0E9EAF1E0DE01509601900D92E7
:101A10009A95E1F79CE0E7EBF1E0DE01D8960190C2
:101A20000D929A95E1F79BE0E4E5F1E0DE01AC5B15
:101A3000BF4F01900D929A95E1F796E0EFE5F1E046
:101A4000DE01A759BF4F01900D929A95E1F79AE0F8
:101A5000E5E6F1E0DE01A15BBF4F01900D929A95A2
:101A6000E1F79FE0E3ECF1E0DE01119601900D92C9
:101A70009A95E1F79CE0E2EDF1E0DE019C960190A1
:101A80000D929A95E1F796E0EEEDF1E0DE01AD59A9
:101A9000BF4F01900D929A95E1F7A89590E08A309A
:101AA000910508F06CC0FC01E85AFF4F0C94C74345
:101AB000CE01875A9F4F7C0102E02FE130E04FEFCB
:101AC0005FEF62E870E014C0CE014E9609C0CE010F
:101AD000409606C0CE01C89603C0CE018C5B9F4FD6
:101AE0007C0102E02FE130E04FEF5FEF68E770E04C
:101AF00088E090E042C0CE0187599F4F7C0102E010
:101B00002FE130E04FEF5FEF6EE670E088E290E0AB
:101B100025D8CE01815B9F4F7C012FE130E04FEF54
:101B20005FEF67E870E08FE090E027C0CE0101969C
:101B30007C0102E02FE130E04FEF5FEF68E770E0FB
:101B400082E090E01AC0CE018C967C0102E02FE189
:101B500030E04FEF5FEF6EE670E084E190E00E94CE
:101B6000AE05CE018D599F4F7C012FE130E04FEF44
:101B70005FEF67E870E08CE390E00E94AE05C25929
:101B8000DF4F0FB6F894DEBF0FBECDBFDF91CF9110
:101B90000F91FF90EF900895CF92DF92EF92FF9216
:101BA0000F931F93A89500EE17E021E430E048EC76
:101BB00050E06AEA70E085E090E00E94B9040FEF1F
:101BC0001FEF21E430E048EC50E063E270E085E094
:101BD00090E04EDA87E5E82E83E0F82E01E02FE171
:101BE00030E040EE57E06CE370E088E290E00E9465
:101BF000AE050FEF1FEF20E530E040E550E065E077
:101C000070E08BEE90E034DA90EEC92E97E0D92E9A
:101C100024E1E22EF12C03E111E026E430E041E37F
:101C200051E066E470E085EF90E0CEDA37E1E32E34
:101C3000F12C24E430E04FE251E064E470E087EFFF
:101C400090E0C2DA0FEF1FEF20E530E040E550E012
:101C500064E670E08BEE90E00BDA45EAE42EF12CBE
:101C600003E111E023E730E041E351E063E770E096
:101C700085EF90E0A9DA53EAE52EF12C25E730E074
:101C80004FE251E065E770E087EF90E09DDA63E9AD
:101C9000E62E65E0F62E02E020EE37E040E050E070
:101CA00068EC70E08DE290E00E94AE051F910F910C
:101CB000FF90EF90DF90CF900895CF92DF92EF9258
:101CC000FF920F931F93CF93DF93CDB7DEB7659746
:101CD0000FB6F894DEBF0FBECDBFA8958FE0E3EC42
:101CE000F1E0DE01119601900D928A95E1F786E010
:101CF000E4EEF1E0DE01509601900D928A95E1F755
:101D000000EE17E021E430E048EC50E06AEA70E0D1
:101D100085E090E00E94B9040FEF1FEF21E430E06E
:101D200048EC50E063E270E085E090E0A1D9CE019C
:101D300001967C0101E02FE130E040EE57E06CE3DA
:101D400070E088E290E00E94AE050FEF1FEF20E503
:101D500030E040E550E065E070E08BEE90E088D93F
:101D600080EEC82E87E0D82E94E1E92EF12C03E115
:101D700011E026E430E041E351E066E470E085EFF5
:101D800090E022DA27E1E22EF12C24E430E04FE269
:101D900051E064E470E087EF90E016DA0FEF1FEF98
:101DA00020E530E040E550E064E670E08BEE90E046
:101DB0005FD935EAE32EF12C03E111E023E730E0AF
:101DC00041E351E063E770E085EF90E0FDD943EA3D
:101DD000E42EF12C25E730E04FE251E065E770E0BA
:101DE00087EF90E0F1D9CE0140967C0102E020EE31
:101DF00037E040E050E068EC70E08DE290E00E9457
:101E0000AE0565960FB6F894DEBF0FBECDBFDF916D
:101E1000CF911F910F91FF90EF90DF90CF90089599
:101E2000CF92DF92EF92FF920F931F93A89500EE4F
:101E300017E021E430E048EC50E06AEA70E085E029
:101E400090E00E94B9040FEF1FEF21E430E048EC6E
:101E500050E063E270E085E090E00AD982E3E82E8A
:101E600085E0F82E01E02FE130E040EE57E06CE332
:101E700070E088E290E00E94AE050FEF1FEF20E5D2
:101E800030E040E550E065E070E08BEE90E0F0D8A7
:101E900090EEC92E97E0D92E24E1E22EF12C03E139
:101EA00011E026E430E041E351E066E470E085EFC4
:101EB00090E08AD937E1E32EF12C24E430E04FE2C0
:101EC00051E064E470E087EF90E07ED90FEF1FEF00
:101ED00020E530E040E550E064E670E08BEE90E015
:101EE000C7D845EAE42EF12C03E111E023E730E006
:101EF00041E351E063E770E085EF90E065D953EA94
:101F0000E52EF12C25E730E04FE251E065E770E087
:101F100087EF90E059D964EAE62E65E0F62E02E0FC
:101F200020EE37E040E050E068EC70E08DE290E0B9
:101F30000E94AE051F910F91FF90EF90DF90CF9020
:101F40000895CF93DF9300D000D0CDB7DEB7809156
:101F5000630080FD57C01C821B821A821982BE0159
:101F60006F5F7F4FCE0103960E9426428B819C813A
:101F70008431954068F489819A81843A964040F48E
:101F800089819A818D32914018F082E080938A068F
:101F90008B819C818937954090F08B819C81843C1A
:101FA000994068F489819A81843A964040F4898105
:101FB0009A818D32914018F083E080938A068B815C
:101FC0009C8189329A4068F089819A8184379E4049
:101FD00040F489819A81813D974018F081E0809397
:101FE0008A068B819C81863F994060F48B819C811D
:101FF0008134964038F089819A81813D974010F074
:1020000010928A0680918A060F900F900F900F9081
:10201000DF91CF910895CF92DF92EF92FF920F93CD
:102020001F93CF93DF9300D000D000D0CDB7DEB7A1
:10203000A89586E0E4EEF1E0DE01119601900D92A4
:102040008A95E1F700EE17E021E430E048EC50E03B
:102050006AEA70E085E090E00E94B9040FEF1FEF9C
:1020600021E430E048EC50E063E270E085E090E08D
:102070000E94380820E530E040E550E065E070E07F
:102080008BEE90E00E943808F0EECF2EF7E0DF2EC6
:10209000A4E1EA2EF12C03E111E026E430E041E373
:1020A00051E066E470E085EF90E08ED8B7E1EB2E6A
:1020B000F12C24E430E04FE251E064E470E087EF7B
:1020C00090E082D80FEF1FEF20E530E040E550E0D0
:1020D00064E670E08BEE90E00E94380815EAE12E8D
:1020E000F12C03E111E023E730E041E351E063E745
:1020F00070E085EF90E068D883EAE82EF12C25E7C0
:1021000030E04FE251E065E770E087EF90E05CD8A7
:10211000CE0101967C0102E020EE37E040E050E085
:1021200068EC70E08CE390E00E94AE058091680658
:10213000811148C0E091C0068E2F90E08830910553
:1021400008F040C0FC01EE59FF4F0C94C743E4E88F
:10215000EE2EE5E0FE2E04C07FE7E72E75E0F72EB9
:1021600002E02FE130E04FEF5FEF65E070E086E4E2
:1021700090E026C065E7E62E65E0F62E18C05BE627
:10218000E52E55E0F52E13C041E6E42E45E0F42E91
:102190000EC037E5E32E35E0F32E09C02DE4E22E24
:1021A00025E0F22E04C093E4E92E95E0F92E02E03A
:1021B0002FE130E04FEF5FEF65E070E08EE190E0FF
:1021C0000E94AE0580916806813001F580916E060F
:1021D000813069F038F08230C9F411E6E12E15E063
:1021E000F12E09C085E7E82E85E0F82E04C00BE645
:1021F000E02E05E0F02E02E02FE130E04FEF5FEF40
:1022000065E070E08EE190E00E94AE058091680686
:10221000823001F580917506813069F038F08230A6
:10222000C9F4F1E6EF2EF5E0FF2E09C0B5E7EB2E7D
:10223000B5E0FB2E04C0ABE6EA2EA5E0FA2E02E0E4
:102240002FE130E04FEF5FEF65E070E08EE190E06E
:102250000E94AE0580916806843001F58091CA061F
:10226000813069F038F08230C9F461E6E62E65E02D
:10227000F62E09C0E5E7EE2EE5E0FE2E04C07BE673
:10228000E72E75E0F72E02E02FE130E04FEF5FEF31
:1022900065E070E08EE190E00E94AE0580916806F6
:1022A000853001F58091BF06813069F038F08230C9
:1022B000C9F431E6E32E35E0F32E09C055E7E52EEB
:1022C00055E0F52E04C04BE6E42E45E0F42E02E086
:1022D0002FE130E04FEF5FEF65E070E08EE190E0DE
:1022E0000E94AE0580916806863001F58091BC069B
:1022F000813069F038F08230C9F481E6E82E85E05B
:10230000F82E09C025E7E22E25E0F22E04C09BE658
:10231000E92E95E0F92E02E02FE130E04FEF5FEF7C
:1023200065E070E08EE190E00E94AE0526960FB663
:10233000F894DEBF0FBECDBFDF91CF911F910F91FB
:10234000FF90EF90DF90CF900895EF92FF920F9360
:102350001F9380916006909161060A97A8F480917E
:10236000370681110CC00FE110E02CE330E044E6A9
:1023700050E06BE470E08EE690E00E94B90481E0EA
:1023800080933706109269068091600690916106ED
:102390000A978A359105A8F48091690681110CC0CD
:1023A0000FE110E02CE330E044E650E06BE470E035
:1023B0008EE690E00E94B90481E080936906109255
:1023C0003706809160069091610684369105A0F0F1
:1023D00080916906813061F40FE110E02CE330E078
:1023E00044E650E06BE470E08EE690E00E94B904B1
:1023F000109269061092370680916706813079F451
:10240000E0906006F090610603E02FE130E04FEFCE
:102410005FEF64E670E082E890E00E94F40580914E
:10242000670681110FC0E0906006F090610603E03E
:102430002FE130E040E058EF64E670E082E890E0A1
:102440000E94F4051F910F91FF90EF900895EF9275
:10245000FF920F931F9380918E0690918F060A979B
:10246000A8F480915F06811111C00FE110E028E20D
:1024700030E048E550E06FEA70E088E090E00E94CC
:10248000B90481E080935F061092BD0680918E06AC
:1024900090918F0684369105D8F4809160069091D2
:1024A00061060A97A8F08091BD06811111C00FE165
:1024B00010E028E230E048E550E06FEA70E088E0A4
:1024C00090E00E94B90481E08093BD0610925F06FF
:1024D00080918E0690918F0684369105A0F08091B0
:1024E000BD06813061F40FE110E028E230E048E5FC
:1024F00050E06FEA70E088E090E00E94B90410922A
:10250000BD0610925F06E0908E06F0908F0602E006
:102510002FE130E04FEF5FEF6EEB70E08EE190E087
:102520000E94F4051F910F91FF90EF900895EF9294
:10253000FF920F931F9380917D068A30A8F48091BB
:10254000660681110CC00FE110E024E230E04AE59C
:1025500050E064E670E088E090E00E94B90481E019
:10256000809366061092790680917D068A508A359E
:10257000A8F48091790681110CC00FE110E024E2EB
:1025800030E04AE550E064E670E088E090E00E94C8
:10259000B90481E0809379061092660680917D06E9
:1025A0008436A1F480917906813061F40FE110E066
:1025B00024E230E04AE550E064E670E088E090E034
:1025C0000E94B904109266061092790680917D06E9
:1025D000843618F084E680937D06E0907D06F12C29
:1025E00002E02FE130E04FEF5FEF6EE670E084E154
:1025F00090E00E94F4058091CB068A30A8F4809187
:10260000C606811111C00FE110E024E230E04AE576
:1026100050E064E670E08FED90E00E94B90481E044
:102620008093C606109290068091CB068A508A3518
:10263000A8F480919006811111C00FE110E024E20E
:1026400030E04AE550E064E670E08FED90E00E94F3
:10265000B90481E0809390061092C6068091CB0663
:10266000843629F41092C6061092900602C0843671
:1026700018F084E68093CB06E090CB06F12C02E0C4
:102680002FE130E04FEF5FEF6EE670E089EE90E013
:102690000E94F4051F910F91FF90EF9008957F9293
:1026A0008F929F92AF92BF92CF92DF92EF92FF9262
:1026B0000F931F93CF93DF93EC016B015A014901F4
:1026C000702EA89580913A0690913B060A97A8F43F
:1026D0008091C106811111C00FE110E02EE130E0C0
:1026E00044E650E065507109CE0144970E94B90458
:1026F00081E08093C1061092830680913A06909102
:102700003B060A978A359105C0F4809183068111B2
:1027100014C00FE110E02EE130E044E650E0B601D5
:1027200065507109CE0144970E94B90481E08093FD
:1027300083061092C1061092620680913A0690912B
:102740003B0684369105C0F080916206811114C069
:102750000FE110E02EE130E044E650E0B6016550B4
:102760007109CE0144970E94B90481E0809362060A
:10277000109283061092C106E0903A06F0903B0654
:10278000072D9401A501B601CE010E94F405A8957C
:10279000DF91CF911F910F91FF90EF90DF90CF903D
:1027A000BF90AF909F908F907F900895CF92DF92CF
:1027B000EF92FF920F931F938FE190E00E942E06FD
:1027C000A89500EE17E021E430E048EC50E06AEA1A
:1027D00070E085E090E00E94B9040FEF1FEF21E464
:1027E00030E048EC50E063E270E085E090E00E9469
:1027F000380885E2E82E83E0F82E01E02FE130E092
:1028000040EE57E06CE370E088E290E00E94AE0595
:102810000FEF1FEF20E530E040E550E065E070E0AD
:102820008BEE90E00E94380890EEC92E97E0D92EEA
:1028300024E1E22EF12C03E111E026E430E041E353
:1028400051E066E470E085EF90E00E94E40837E133
:10285000E32EF12C24E430E04FE251E064E470E038
:1028600087EF90E00E94E4080FEF1FEF20E530E0D3
:1028700040E550E064E670E08BEE90E00E9438089E
:1028800045EAE42EF12C03E111E023E730E041E3D7
:1028900051E063E770E085EF90E00E94E40853EABE
:1028A000E52EF12C25E730E04FE251E065E770E0DE
:1028B00087EF90E00E94E40863E9E62E65E0F62EDB
:1028C00002E020EE37E040E050E068EC70E08DE29E
:1028D00090E00E94AE058FE19EE40197F1F700C001
:1028E00000001F910F91FF90EF90DF90CF9008951F
:1028F000A89583EB92E00E94E246813071F4A49A9D
:1029000080E185BBA8952FEF82E597E021508040BC
:102910009040E1F700C0000015BAA8950895A89569
:1029200083EB92E00E94E246813021F5A49A80E197
:1029300085BB2FEF32E597E0215030409040E1F722
:1029400000C00000A89515BA2FEF32E597E021509E
:1029500030409040E1F700C00000A89585BB2FEF04
:1029600032E587E0215030408040E1F700C00000B0
:10297000A89515BA0895A89583EB92E00E94E246C7
:10298000813009F048C0A49A80E185BBA8952FEF5B
:1029900032E597E0215030409040E1F700C0000060
:1029A000A89515BAA8952FEF32E597E02150304051
:1029B0009040E1F700C00000A89585BBA8952FEFD7
:1029C00032E597E0215030409040E1F700C0000030
:1029D000A89515BAA8952FEF32E597E02150304021
:1029E0009040E1F700C00000A89585BB2FEF32E5CD
:1029F00087E0215030408040E1F700C00000A895FA
:102A000015BA9FEF22E537E0915020403040E1F7C2
:102A100000C00000A89508951092CB06BC9A809142
:102A2000CB06880F81BF10927D06139A80917D0698
:102A3000880F809386009FDF8DE490E09093C3061B
:102A40008093C2060895A89510927E061092720691
:102A5000109235061092930610926F06109265063A
:102A600010927F061092780610928D06109236060C
:102A7000A89584EB92E00E94EA46909374068093B6
:102A80007306A8958091680681112AC0A895E091E7
:102A9000C0068E2F90E08830910510F5FC01E659B4
:102AA000FF4F4EE150E00C94C74364E972E014C05C
:102AB00066E772E011C068E572E00EC06AE372E09A
:102AC0000BC06CE172E008C06EEF71E005C060EE13
:102AD00071E002C062EC71E080E496E00E94D246B0
:102AE000A895809168068130D1F4A89580916E06F2
:102AF000813069F038F0823091F44EE150E068E6C0
:102B000071E009C04EE150E064EA71E004C04EE1BA
:102B100050E066E871E080E496E00E94D246A89515
:102B2000809168068230D1F4A89580917506813035
:102B300069F038F0823091F44EE150E06EE071E0DF
:102B400009C04EE150E06AE471E004C04EE150E09B
:102B50006CE271E080E496E00E94D246A8958091F4
:102B600068068430C9F48091CA06813069F038F073
:102B7000823091F44EE150E064EB70E009C04EE128
:102B800050E060EF70E004C04EE150E062ED70E0B4
:102B900080E496E00E94D246A89580916806853030
:102BA000C9F48091BF06813069F038F0823091F429
:102BB0004EE150E06AE570E009C04EE150E066E9A0
:102BC00070E004C04EE150E068E770E080E496E019
:102BD0000E94D246A895809168068630C9F48091FB
:102BE000BC06813069F038F0823091F44EE150E05B
:102BF00060E070E009C04EE150E06CE370E004C0BA
:102C00004EE150E06EE170E080E496E00E94D24632
:102C1000A89587EC90E00197F1F700C00000809143
:102C20004006909141069093320680933106809140
:102C3000420690914306909382068093810680918C
:102C400044068093C8068091460680936D06809165
:102C500048068093950680914A0680936C06809181
:102C60004C0680937B0680914E0680937A06809175
:102C7000500680932D0680915206909153069093B2
:102C8000B9068093B806809154068093940680918B
:102C90006806873021F480915606809368068091FB
:102CA0005806909159069093B7068093B606809186
:102CB0005A0690915B0690933F0680933E06809162
:102CC0005C0690915D069093640680936306A895D8
:102CD000089580919306811117C020916C06809110
:102CE000600690916106821B9109029768F482E365
:102CF0008093CB0681E08093930680936506809154
:102D00009506811101C0F4DD20916C0630E06091E0
:102D1000C8064091C4065091C506649FC001659FD6
:102D2000900D11246AE070E00E94B343620F731F9C
:102D30007093300660932F069091CB064091310638
:102D4000509132064617570720F4509330064093AF
:102D50002F0680917B06891710F48093CB06809113
:102D60006006909161062817390720F04817590727
:102D700028F155C020918D062111F8CF84179507B1
:102D8000A8F760912F06709130062091CB06861728
:102D9000970750F42F5F253618F42093CB06E6CF23
:102DA00024E62093CB0687C0222319F021502093DC
:102DB000CB062091CB062223C9F27DC02091CB0601
:102DC000222319F021502093CB06841B950B0697E4
:102DD00068F08091CB068A3010F41092CB06809177
:102DE000CB068A3018F08A508093CB068091360645
:102DF000811106C094DD81E08093780680933606C9
:102E000020913C0630913D068091730690917406A6
:102E10008217930720F400DE81E08093670680919B
:102E20006F0681114FC04091B6065091B706809150
:102E30006C0690E08417950708F044C0E0916006A6
:102E4000F09161064E175F0729F481E080938D06AB
:102E500080937F0680918D068130A1F560913806C0
:102E60007091390620913E0630913F066217730734
:102E700078F48091CB06E417F50728F48F5F853648
:102E800028F084E603C0882319F081508093CB0694
:102E900026173707B8F410928D068091C4069091DA
:102EA000C506821B930B9093C5068093C40681E0F0
:102EB00080936F0608954817590708F0B0CF209106
:102EC000CB0680CF089580919306811117C0809121
:102ED0006C0690E02091600630916106821793079E
:102EE00068F482E38093CB0681E08093930680931D
:102EF000650680919506811101C0FADCE0916C06AF
:102F0000F0E04091C8062091C4063091C506429F6A
:102F1000C001439F900D11246AE070E00E94B3430A
:102F20006E0F7F1F7093300660932F069091CB0633
:102F300040913106509132064617570720F45093BE
:102F4000300640932F0680917B06891710F48093FA
:102F5000CB062091600630916106E217F307D0F4AA
:102F600080918D06811116C02417350798F4609161
:102F70002F06709130068091CB062617370728F46C
:102F80008F5F853628F084E603C0882319F08150CE
:102F90008093CB064217530770F58091CB06815082
:102FA0008093CB06241B350B2630310558F08A3030
:102FB00010F41092CB068091CB068A3018F08A501C
:102FC0008093CB0680913606811106C0A8DC81E093
:102FD000809378068093360620913C0630913D061A
:102FE00080917306909174068217930720F414DD84
:102FF00081E08093670680916F06811146C0409101
:10300000B6065091B70680916C0690E0841795073C
:10301000E0F5E0916006F09161064E175F0729F434
:1030200081E080938D0680937F0680918D068130AC
:1030300061F5609138067091390620913E06309115
:103040003F066217730778F48091CB06E417F50703
:1030500028F48F5F853628F084E603C0882319F0B2
:1030600081508093CB062617370778F410928D068F
:103070008091C4069091C506821B930B9093C50660
:103080008093C40681E080936F06089540916D0699
:1030900020913A0630913B06429FC001439F900D1C
:1030A00011246AE070E00E94B3437093920660932B
:1030B000910680917D06853618F084E680937D0622
:1030C00090917A0680917D06981710F490937D0672
:1030D00080917E0620918E0630918F0681110DC061
:1030E0002639310520F484E680937D0606C0263912
:1030F000310519F081E080937E0680917E06409133
:103100008106509182068130D9F464177507C0F4A6
:1031100080917D062617370770F48F5F981718F097
:1031200080937D0602C090937D0680917D06853652
:1031300038F084E603C0882319F0815080937D061F
:103140004617570768F52417350770F480917D06F8
:103150008F5F853608F084E680937D0680917D063A
:10316000981710F490937D0642175307C8F4809186
:103170007D06882319F0815080937D06C901841B48
:10318000950B0B9768F080917D068A3010F41092B1
:103190007D0680917D068A3018F08A5080937D06E6
:1031A00080917B069091CB06891710F48093CB0613
:1031B0004217530740F48091CB068F5F853608F0A5
:1031C00084E68093CB06089540916D0620913A06DF
:1031D00030913B06429FC001439F900D11246AE04D
:1031E00070E00E94B34370939206609391068091C1
:1031F0007D06853618F084E680937D0690917A06E8
:1032000080917D06981710F490937D0680917E063C
:10321000811111C020918E0630918F06263931051B
:1032200020F484E680937D0606C02639310519F026
:1032300081E080937E0680917E06409181065091C8
:1032400082068130F9F464177507E0F420918E0648
:1032500030918F0680917D062617370770F48F5FB7
:10326000981718F080937D0602C090937D06809198
:103270007D06853638F084E603C0882319F0815036
:1032800080937D064617570788F520918E0630916A
:103290008F062417350770F480917D068F5F853681
:1032A00008F084E680937D0680917D06981710F4DF
:1032B00090937D0642175307C8F480917D068823BA
:1032C00019F0815080937D06241B350B2B3031057E
:1032D00068F080917D068A3010F410927D0680910E
:1032E0007D068A3018F08A5080937D060895CF932A
:1032F000C0919506C130C9F480917206811115C044
:1033000080916C0690E0209160063091610628174C
:10331000390758F080918E0690918F06909334066D
:1033200080933306E5DAC093720640916D062091D2
:103330003A0630913B06429FC001439F900D1124F5
:103340006AE070E00E94B343709392066093910626
:1033500080917D06853618F084E680937D06809105
:103360007E06811111C080918E0690918F06843661
:10337000910520F484E680937D0606C0843691058D
:1033800019F081E080937E0680917E06C0917206DE
:10339000813051F5C11128C080918106909182063B
:1033A0006817790708F047C020918E0630918F0684
:1033B00080917D062617370788F48F5F80937D06FE
:1033C00090917A06981710F490937D0680917D066F
:1033D000853688F184E680937D0606C0882359F1FE
:1033E000815080937D0627C0C13029F58091330636
:1033F000909134060E94083CC093780680913C0668
:1034000090913D06CD97B8F080916C0690E02091A8
:103410006006309161062817390748F48091330619
:10342000909134060A969093340680933306109256
:103430003D0610923C068091810690918206209173
:103440009106309192068217930748F420919506D1
:10345000211105C08A559109CF910C94083CCF9158
:103460000895BC9A8091CB06880F81BF139A8091F2
:103470007D06880F8093860080916806811102C0C6
:1034800036DF27DC80916806813019F410927D06C2
:103490001ADD80916806823019F41092CB0627DF7E
:1034A00080916806833011F40E944C3C809168063C
:1034B000843009F4EBDD80916806853009F4E6DD9F
:1034C00080916806863009F47FDE80916806893035
:1034D00069F480918E0690918F060E94CD3B809179
:1034E0007D06863518F081E080936706089563ECC9
:1034F00070E084E992E00E94054762EC71E086E9A1
:1035000092E00E94054766E170E088E992E00E943F
:10351000054766E170E08AE992E00E94054761E0B4
:1035200070E08CE992E00E940547A8956EE670E095
:103530008EE992E00E94054764E670E080EA92E03E
:103540000E94054764E670E082EA92E00E94054727
:1035500060E070E084EA92E00E940547A89560E090
:1035600070E086EA92E00E94054760E070E088EA39
:1035700092E00E94054760E070E08AEA92E00E94D3
:10358000054760E070E08CEA92E00E94054760E049
:1035900070E08EEA92E00E94054760E070E080EB08
:1035A00092E00E940547A89566EE70E086E792E0FB
:1035B0000E94054762EC71E088E792E00E940547AF
:1035C00066E170E08AE792E00E94054766E170E0FC
:1035D0008CE792E00E94054761E070E08EE792E0A0
:1035E0000E940547A89563E770E080E892E00E949A
:1035F000054764E670E082E892E00E94054764E6D1
:1036000070E084E892E00E94054760E070E086E8A0
:1036100092E00E94054760E070E088E892E00E9436
:10362000054760E070E08AE892E00E940547A895AF
:1036300060E070E08CE892E00E94054760E070E096
:103640008EE892E00E94054760E070E080E992E039
:103650000E94054760E070E082E992E00E94054721
:10366000A89566EE70E088E592E00E94054762EC5E
:1036700071E08AE592E00E94054766E170E08CE522
:1036800092E00E94054766E170E08EE592E00E94BC
:10369000054761E070E080E692E00E940547A8954A
:1036A00063E770E082E692E00E94054764E670E01E
:1036B00084E692E00E94054764E670E086E692E0C8
:1036C0000E94054760E070E088E692E00E940547AE
:1036D00060E070E08AE692E00E94054760E070E0FA
:1036E0008CE692E00E940547A89560E070E08EE6C7
:1036F00092E00E94054760E070E080E792E00E945F
:10370000054760E070E082E792E00E94054760E0D4
:1037100070E084E792E00E940547A89566E970E0B2
:103720008AE392E00E94054768EC70E08CE392E047
:103730000E94054766E170E08EE392E00E94054733
:1037400066E170E080E492E00E94054761E070E08D
:1037500082E492E00E940547A89563E770E084E464
:1037600092E00E94054764E670E086E492E00E94E1
:10377000054764E670E088E492E00E94054760E057
:1037800070E08AE492E00E94054760E070E08CE41B
:1037900092E00E94054760E070E08EE492E00E94B3
:1037A0000547A89560E070E080E592E00E9405473B
:1037B00060E070E082E592E00E94054760E070E022
:1037C00084E592E00E94054760E070E086E592E0C3
:1037D0000E940547A8956EEB70E08CE192E00E9494
:1037E000054768EC70E08EE192E00E94054766E1D3
:1037F00070E080E292E00E94054766E170E082E2BC
:1038000092E00E94054761E070E084E292E00E944D
:103810000547A89564E670E086E292E00E940547BD
:1038200064E670E088E292E00E94054764E670E09A
:103830008AE292E00E94054760E070E08CE292E04C
:103840000E94054760E070E08EE292E00E9405472A
:1038500060E070E080E392E00E940547A89560E098
:1038600070E082E392E00E94054760E070E084E34C
:1038700092E00E94054760E070E086E392E00E94DB
:10388000054760E070E088E392E00E940547A89554
:1038900066EE70E08EEF91E00E94054762EC71E009
:1038A00080E092E00E94054766E170E082E092E0ED
:1038B0000E94054766E170E084E092E00E940547BF
:1038C00061E070E086E092E00E940547A89563E71A
:1038D00070E088E092E00E94054764E670E08AE0CC
:1038E00092E00E94054764E670E08CE092E00E945E
:1038F000054760E070E08EE092E00E94054760E0DE
:1039000070E080E192E00E94054760E070E082E1B3
:1039100092E00E940547A89560E070E084E192E0A3
:103920000E94054760E070E086E192E00E94054752
:1039300060E070E088E192E00E94054760E070E09E
:103940008AE192E00E940547A89566EE70E080EE5D
:1039500091E00E94054762EC71E082EE91E00E94E6
:10396000054766E170E084EE91E00E94054766E15C
:1039700070E086EE91E00E94054761E070E088EE1D
:1039800091E00E940547A89563E770E08AEE91E018
:103990000E94054764E670E08CEE91E00E940547C6
:1039A00064E670E08EEE91E00E94054760E070E012
:1039B00080EF91E00E94054760E070E082EF91E0C7
:1039C0000E94054760E070E084EF91E00E940547A7
:1039D000A89560E070E086EF91E00E94054760E006
:1039E00070E088EF91E00E94054760E070E08AEFA8
:1039F00091E00E94054760E070E08CEF91E00E944A
:103A00000547A89563EC70E084EA91E00E940547C1
:103A100066E170E088EA91E00E94054761E070E0AD
:103A20008CEA91E00E9405476FE070E08EEA91E039
:103A30000E940547A89564E670E080EB91E00E9443
:103A4000054761E070E08AEB91E00E94054763EC76
:103A500070E08CEB91E00E9405476AE070E08EEB2D
:103A600091E00E940547A89562EC71E08CE491E03A
:103A70000E94054766E170E080E591E00E940547FD
:103A800061E070E082E591E00E9405476EE670E03B
:103A900084E591E00E940547A89564E670E088E51A
:103AA00091E00E94054762E070E080E691E00E94AC
:103AB000054762EC71E082EF90E00E94054766E105
:103AC00070E084EF90E00E94054762E170E086EFCD
:103AD00090E00E940547A89564E670E08CEF90E0C6
:103AE0000E94054764E670E08EEF90E00E94054773
:103AF00064E070E086E091E00E9405476CE271E0CE
:103B00008CE091E00E940547A89562EC71E088E99D
:103B100090E00E94054766E170E08AE990E00E942B
:103B2000054766E170E08CE990E00E94054761E09E
:103B300070E08EE990E00E940547A8956EE670E07F
:103B400080EA90E00E94054764E670E082EA90E037
:103B50000E94054764E670E084EA90E00E94054711
:103B600065E070E08CEA90E00E940547A89562EC61
:103B700071E08EE390E00E94054766E170E082E428
:103B800090E00E94054761E070E084E490E00E94CC
:103B900005476EE670E086E490E00E940547A89530
:103BA00064E670E08AE490E00E94054766E070E019
:103BB00082E590E00E94054763EC70E084E992E0C2
:103BC0000E940547A89508956FE070E088EB92E0A9
:103BD0000E9405476FE070E086EB92E00E94054787
:103BE0006FE070E084EB92E00E94054761E083EBB8
:103BF00092E00E94F84661E082EB92E00C94F84675
:103C00008FB9779BFECF8FB10895CF93A39AAB9ACC
:103C1000AB9880E0F5DFC82F80E0F2DFAB9A6C2F25
:103C200070E0762F6627682B687F7F7723E0769594
:103C300067952A95E1F780E090E00E94C24220E07B
:103C400030E040E85EE30E9428430E949642709371
:103C5000610660936006CB01CF910895CF93A79A38
:103C6000AF9AAF9880E0CCDFC82F80E0C9DFAF9A71
:103C70006C2F70E0762F6627682B687F7F7723E0B4
:103C8000769567952A95E1F780E090E00E94C24220
:103C900020E030E040E85EE30E9428430E94964224
:103CA00070938F0660938E06CB01CF91089580E0CC
:103CB00091E09093D7068093D606809161068F930A
:103CC000809160068F938AEE91E09F938F930E947C
:103CD00002448DE08A95F1F7000080913B068F93B6
:103CE00080913A068F9384EF91E09F938F930E9487
:103CF00002449DE09A95F1F7000080917D061F92A5
:103D00008F938EEF91E09F938F930E9402448DE0FA
:103D10008A95F1F700008091CB061F928F9389E07E
:103D200092E09F938F930E9402449DE09A95F1F751
:103D3000000083E192E09F938F930E9402448DE004
:103D40008A95F1F7000080918F068F9380918E06FF
:103D50008F938BE192E09F938F930E940244A895EA
:103D60008DB79EB746960FB6F8949EBF0FBE8DBF17
:103D700080916706811108C084E292E09F938F933F
:103D80000E9402440F900F90A895809167068130A1
:103D900041F48BE292E09F938F930E9402440F9034
:103DA0000F909DE09A95F1F70000E09168068E2F44
:103DB00090E08830910508F09DC0FC01EE58FF4F5F
:103DC0000C94C74382E392E09F938F930E94024436
:103DD000A8950F900F90E091C0068E2F90E088304C
:103DE000910508F087C0FC01E658FF4F0C94C743CB
:103DF00081E492E071C081E592E06EC089E892E0D2
:103E00006BC088E992E068C087EA92E065C086EB03
:103E100092E09F938F930E940244A8950F900F9079
:103E200080916E06813009F452C008F44DC0823092
:103E300009F450C0089586EC92E09F938F930E94FE
:103E40000244A8950F900F9080917506813009F477
:103E50003EC0D0F1823009F43DC0089587ED92E074
:103E600042C085EE92E09F938F930E940244A895F2
:103E70000F900F908091CA06813049F128F182306D
:103E800049F1089586EF92E09F938F930E94024438
:103E9000A8950F900F908091BF068130C1F0A0F0DF
:103EA0008230C1F0089589E093E09F938F930E9440
:103EB0000244A8950F900F908091BC06813039F094
:103EC00018F0823039F008958CE592E005C08BE659
:103ED00092E002C08AE792E09F938F930E9402448F
:103EE00007C08BE193E09F938F930E940244A895B3
:103EF0000F900F900895CF92DF92EF92FF920F9361
:103F00001F93CF93DF9300D000D0CDB7DEB7809161
:103F10006706813009F034C180917606909177066A
:103F2000892BD9F40FE110E024E230E04AE550E0BB
:103F300064E670E088E090E00E94B90424E230E09A
:103F40004AE550E064E670E08FED90E00E94B9042D
:103F5000A895A49AAC980E942B0CCC24C394D12C85
:103F600080916706813009F00BC1A895A0DE809191
:103F7000C2069091C3068A35910549F42FEF8DE36F
:103F800099E4215080409040E1F700C00000A895DE
:103F900003E02FE130E04FEF5FEF69E170E085E88B
:103FA00090E00E944F138091630080FD81C0A8952E
:103FB0001C821B821A821982BE016F5F7F4FCE0165
:103FC00003960E9426428B819C818431954088F41F
:103FD00089819A81883D9E4060F489819A81853CDF
:103FE000994038F0D0927706C092760610928506F6
:103FF00013D48B819C818431954098F589819A8175
:104000008C3D954070F589819A81853F914048F1BA
:10401000D0927706C0927606109296068091680636
:10402000811102C00E94803180916806813011F4B4
:104030000E946C3480916806823011F40E947335BE
:1040400080916806843011F40E947A368091680667
:10405000853009F4AED480916806863011F40E9450
:10406000783080912C06813019F58B819C81853CBC
:104070009940F0F089819A818C3D9540C8F48981FE
:104080009A81853F9140A0F0D0927706C092760643
:104090000E94D61380E00E948C3A0E94F63A109259
:1040A0007706109276068FE190E00E942E0623DFBD
:1040B000ACDD0E94A511A8958FEF91EE24E0815010
:1040C00090402040E1F700C00000C8DDA8950E94A4
:1040D0002712E0907D06F12C02E02FE130E04FEF57
:1040E0005FEF6EE670E08CE190E00E94F405E090F6
:1040F000CB06F12C2FE130E04FEF5FEF6EE670E082
:1041000080EF90E00E94F40580912C06813011F43C
:104110000E947E3B0E94610B80916706811120CF37
:10412000A8950E942315A8950E947814A8950E942E
:104130002B0C0FE110E029E130E04AE550E06EE69B
:1041400070E088E090E00E94B90429E130E04AE59F
:1041500050E06EE670E08FED90E00E94B90480912F
:104160002C06813021F40E94863A0E94B83B1092BE
:104170003B0610923A061092770610927606F0CE21
:104180000F900F900F900F90DF91CF911F910F9193
:10419000FF90EF90DF90CF900895EF92FF920F93F2
:1041A0001F93CF93DF9380918406813009F047C13C
:1041B0008FE190E00E942E060E945D0E85E08093C4
:1041C0008A06C5E080918406813009F038C10E94DA
:1041D000A10F80918A068230D9F48091B5068F5F55
:1041E0008093B5060FE110E02CE330E046EE50E09E
:1041F00069E670E081E090E00E94B90422E330E0DB
:1042000043EC50E068E270E088E090E00E94B9047E
:1042100080918A068330D9F48091B50681508093CD
:10422000B5060FE110E02CE330E046EE50E069E621
:1042300070E081E090E00E94B90422E330E043ECBA
:1042400050E068E270E088E090E00E94B90480915C
:10425000B506853010F01092B5068091B506823013
:1042600081F1B8F48823D9F0813009F0C1C073EE30
:10427000E72E75E0F72E01E02FE130E04FEF5FEF22
:104280006CE370E088E090E00E94AE0586EB92E07F
:1042900029C08330B1F1843009F471C0A9C0ECEFBA
:1042A000EE2EE5E0FE2E01E02FE130E04FEF5FEF74
:1042B0006CE370E08FE090E00E94AE0588EB92E046
:1042C00011C067EDE62E65E0F62E01E02FE130E04B
:1042D0004FEF5FEF6CE370E082E390E00E94AE0589
:1042E00084EB92E00E94EA467C0103E02FE130E09B
:1042F0004FEF5FEF62E870E080E590E00E94F40528
:1043000077C04FEBE42E45E0F42E01E02FE130E0E2
:104310004FEF5FEF6CE370E088E290E00E94AE0543
:104320005DECE52E55E0F52E02E02FE130E04FEF99
:104330005FEF62E870E088E290E00E94AE05809155
:104340008A06811119C0D3D83FDC39E8E32E35E065
:10435000F32E2FE130E04FEF5FEF62E870E088E28C
:1043600090E00E94AE052FEF89E698E12150804051
:104370009040E1F700C00000C0938A0639C02EEAE1
:10438000E22E25E0F22E01E02FE130E04FEF5FEF6B
:104390006CE370E08EE190E00E94AE0583EB92E06A
:1043A0000E94E246813079F490EAE92E95E0F92EF8
:1043B00003E02FE130E04FEF5FEF62E870E080E56F
:1043C00090E00E94AE0583EB92E00E94E2468111EC
:1043D0000FC08BE9E82E85E0F82E03E02FE130E0F6
:1043E0004FEF5FEF62E870E080E590E00E94AE057D
:1043F000D0918A06D13069F4109284061092770623
:10440000109276068FE190E00E942E06D093670608
:1044100072DD80918A06811106C081E08093840656
:104420001092C70613D0C0938A062FE785EB91E060
:10443000215080409040E1F700C00000C3CEDF91E2
:10444000CF911F910F91FF90EF900895BF92CF925F
:10445000DF92EF92FF920F931F93CF93DF938091A0
:10446000C7068111CFC185E080938A06C9E1D0E0FB
:1044700025E0C22ED12C35E0B32E8091C7068111E4
:10448000C1C18091B506813009F46FC038F0823027
:1044900009F4DDC0843009F441C1A4C188EB92E085
:1044A0000E94EA467C0103E02FE130E040E058EF53
:1044B00062E870E080E590E00E94F40588EB92E00D
:1044C0000E94EA4690938906809388060E94A10F75
:1044D00080918A068230A9F480918806909189069D
:1044E000019690938906809388060FE110E02CE3F3
:1044F00030E046EE50E069E670E081E090E00E9436
:10450000B90480918A068330A9F48091880690913D
:104510008906019790938906809388060FE110E041
:104520002CE330E046EE50E069E670E081E090E098
:104530000E94B90480918806909189064A9720F0DC
:10454000D0938906C0938806809188069091890649
:104550000A9720F4D0938906C09388066091880654
:104560007091890688EB92E066C086EB92E00E942B
:10457000EA467C0103E02FE130E040E058EF62E8DA
:1045800070E080E590E00E94F40586EB92E00E94E6
:10459000EA4690936B0680936A060E94A10F809171
:1045A0008A068230A9F480916A0690916B06019682
:1045B00090936B0680936A060FE110E02CE330E0E5
:1045C00046EE50E069E670E081E090E00E94B904B8
:1045D00080918A068330A9F480916A0690916B06D7
:1045E000019790936B0680936A060FE110E02CE32D
:1045F00030E046EE50E069E670E081E090E00E9435
:10460000B90480916A0690916B064A9720F0D09386
:104610006B06C0936A0680916A0690916B060A97B2
:1046200020F4D0936B06C0936A0660916A0670917D
:104630006B0686EB92E00E9405472FE788E391E046
:10464000215080409040E1F700C00000CBC084EBD7
:1046500092E00E94EA467C0103E02FE130E040E076
:1046600058EF62E870E080E590E00E94F40584EB8A
:1046700092E00E94EA4690938706809386060E9405
:10468000A10F80918A068230A9F4809186069091CC
:104690008706019690938706809386060FE110E0C7
:1046A0002CE330E046EE50E069E670E081E090E017
:1046B0000E94B90480918A068330A9F4809186060D
:1046C00090918706019790938706809386060FE165
:1046D00010E02CE330E046EE50E069E670E081E067
:1046E00090E00E94B90480918606909187064F97CA
:1046F00020F0D0928706C09286068091860690911F
:104700008706059720F4D0928706C09286066091AE
:1047100086067091870684EB92E08DCF83EB92E062
:104720000E94E24680932E060E94A10F80918A0685
:10473000823089F480912E068F5F80932E060FE1E0
:1047400010E02CE330E046EE50E069E670E081E0F6
:1047500090E00E94B90480918A06833089F48091A8
:104760002E06815080932E060FE110E02CE330E0FE
:1047700046EE50E069E670E081E090E00E94B90406
:1047800080912E06823010F010922E0680912E0617
:10479000813079F490EAE92E95E0F92E03E02FE1DB
:1047A00030E040E058EF62E870E080E590E00E9481
:1047B000AE0580912E0681110FC08BE9E82E85E0B1
:1047C000F82E03E02FE130E040E058EF62E870E0BF
:1047D00080E590E00E94AE0560912E0683EB92E0AA
:1047E0000E94F84680918A06813049F48093C7067A
:1047F000809384068FE190E00E942E06CEDCB0927A
:104800008A063BCEDF91CF911F910F91FF90EF90E1
:10481000DF90CF90BF9008959F92AF92BF92CF92BA
:10482000DF92EF92FF920F931F93CF93DF938091CC
:1048300085068111B2C08FE190E00E942E060E9491
:10484000CC0D85E080938A0610928406C0E089E052
:10485000E82ED1E097E0D92E26E0C22E35E0F32EE7
:1048600044E0B42E53E0A52E62E0962E809185069A
:10487000811193C00E94A10F80918A06823069F451
:10488000CF5F0FE110E02CE330E046EE50E069E648
:1048900070E081E090E00E94B90480918A06833044
:1048A00069F4C1500FE110E02CE330E046EE50E037
:1048B00069E670E081E090E00E94B904CA3008F037
:1048C000C0E08C2F0E94E00C8C2F90E08A30910584
:1048D000A8F5FC01EE57FF4F0C94C74310928406D5
:1048E000109268062BC010928406D093680626C0EA
:1048F000109284069092680621C010928406A092BD
:1049000068061CC010928406B092680617C0109208
:104910008406F092680612C010928406C09268065F
:1049200004C010928406D0926806C8E007C0D093F5
:10493000840604C010928406E092680680918A067C
:104940008130F9F480918406813049F41092680630
:10495000109285068FE190E00E942E061EDCD09317
:10496000850610927706109276068091680690E090
:1049700090935706809356068FE190E00E942E0692
:10498000BADAF0928A062FEF80E792E02150804059
:104990009040E1F700C0000069CFDF91CF911F91F7
:1049A0000F91FF90EF90DF90CF90BF90AF909F90CE
:1049B0000895EF92FF920F931F93CF93DF93A895E3
:1049C000809196068111F4C08FE190E00E942E063E
:1049D0000E94100F8091BF0690E090937106809323
:1049E000700685E080938A06C1E0D5E08091960646
:1049F0008111DEC0A8950E94A10F80918A068230A5
:104A0000A9F48091700690917106019690937106B9
:104A1000809370060FE110E02CE330E046EE50E0AA
:104A200069E670E081E090E00E94B90480918A0616
:104A30008330A9F48091700690917106019790934C
:104A40007106809370060FE110E02CE330E046EE33
:104A500050E069E670E081E090E00E94B904809146
:104A6000700690917106039720F0109271061092D3
:104A7000700680917006909171068130910589F1E0
:104A8000D0F0029709F046C081E6E82E85E0F82EC6
:104A900002E02FE130E04FEF5FEF6DE770E088E27A
:104AA00090E00E94AE0582E08093BF064EE150E0A8
:104AB0006AE570E02BC025E7E22E25E0F22E02E049
:104AC0002FE130E04FEF5FEF6DE770E088E290E0BC
:104AD0000E94AE051092BF064EE150E066E970E01C
:104AE00015C09BE6E92E95E0F92E02E02FE130E0BB
:104AF0004FEF5FEF6DE770E088E290E00E94AE0557
:104B0000C093BF064EE150E068E770E080E496E0B5
:104B10000E94D24680918A0681110FC0A895C09349
:104B200096061092770610927606C09385068FE15E
:104B300090E00E942E06A895DED980918A068130E9
:104B400059F5A895809396061092770610927606EE
:104B5000809385068FE190E00E942E06A895109222
:104B6000CC068091BF06813069F038F0823091F434
:104B70004EE150E06AE570E009C04EE150E066E9C0
:104B800070E004C04EE150E068E770E080E496E039
:104B90000E94D246A89513D0D0938A062FEF80E7C3
:104BA00092E0215080409040E1F700C000001ECF0D
:104BB000DF91CF911F910F91FF90EF900895EF92A9
:104BC000FF920F931F93CF938091CC0681110C9489
:104BD00072308FE190E00E942E060E940B1085E05B
:104BE00080938A06C5E08091CC0681110C947230C6
:104BF0000E94A10F80918A068230D9F48091BB0671
:104C00008F5F8093BB060FE110E02CE330E046EEAF
:104C100050E069E670E081E090E00E94B90422E390
:104C200030E043EC50E068E270E088E090E00E9401
:104C3000B90480918A068330D9F48091BB068150F3
:104C40008093BB060FE110E02CE330E046EE50E02D
:104C500069E670E081E090E00E94B90422E330E070
:104C600043EC50E068E270E088E090E00E94B90414
:104C70008091BB068E3010F01092BB06E091BB060F
:104C80008E2F90E08E30910510F00C942D2FFC01AA
:104C9000E457FF4F809168060C94C743811137C0D9
:104CA0008091400690914106893E934020F01092F9
:104CB0004106109240067BE1E72E75E0F72E01E0F9
:104CC0002FE130E04FEF5FEF62E370E08FE090E0C4
:104CD0000E94AE05E4E1EE2EE5E0FE2E2FE130E08D
:104CE0004FEF5FEF66E470E08CE390E00E94AE056A
:104CF000E0904006F090410603E02FE130E04FEFF6
:104D00005FEF62E870E080E590E00E94F40580913A
:104D10006806813009F0B6C780914006909141063F
:104D2000893E934020F010924106109240065BE1CC
:104D3000E52E55E0F52E01E02FE130E04FEF5FEF7B
:104D400062E370E08FE090E00E94AE0564E1E62E41
:104D500065E0F62E2FE130E04FEF5FEF66E470E0A4
:104D60008CE390E00E94AE05E0904006F090410692
:104D70007EC7811137C08091420690914306893EDB
:104D8000934020F010924306109242063CEFE32E2F
:104D900034E0F32E01E02FE130E04FEF5FEF62E30C
:104DA00070E08FE090E00E94AE054EEEE42E44E00D
:104DB000F42E2FE130E04FEF5FEF66E470E08CE31C
:104DC00090E00E94AE05E0904206F090430603E0BA
:104DD0002FE130E04FEF5FEF62E870E080E590E0B8
:104DE0000E94F40580916806813031F48091BB0601
:104DF0008F5F8093BB0639C08230B9F5809142063F
:104E000090914306893E934020F010924306109201
:104E100042069CEFE92E94E0F92E01E02FE130E00C
:104E20004FEF5FEF62E370E08FE090E00E94AE052D
:104E30002EEEE22E24E0F22E2FE130E04FEF5FEF76
:104E400066E470E08CE390E00E94AE05E0904206DC
:104E5000F090430603E02FE130E04FEF5FEF62E8B0
:104E600070E080E590E00E94F4058091680684304F
:104E7000B9F58091420690914306893E934020F017
:104E800010924306109242060CEFE02E04E0F02E42
:104E900001E02FE130E04FEF5FEF62E370E08FE081
:104EA00090E00E94AE058EEEE82E84E0F82E2FE111
:104EB00030E04FEF5FEF66E470E08CE390E00E943B
:104EC000AE05E0904206F090430603E02FE130E0AB
:104ED0004FEF5FEF62E870E080E590E00E94F4053C
:104EE000809168068530B9F580914206909143061D
:104EF000893E934020F01092430610924206BCEF88
:104F0000EB2EB4E0FB2E01E02FE130E04FEF5FEF3E
:104F100062E370E08FE090E00E94AE051EEEE12EAD
:104F200014E0F12E2FE130E04FEF5FEF66E470E028
:104F30008CE390E00E94AE05E0904206F0904306BC
:104F400003E02FE130E04FEF5FEF62E870E080E5D3
:104F500090E00E94F40580916806863009F07DC7D4
:104F60008091420690914306893E934020F0109232
:104F7000430610924206FCEFEF2EF4E0FF2E01E014
:104F80002FE130E04FEF5FEF62E370E08FE090E001
:104F90000E94AE05AEEEEA2EA4E0FA2E2FE130E03C
:104FA0004FEF5FEF66E470E08CE390E00E94AE05A7
:104FB000E0904206F0904306B2C5811136C0809160
:104FC0004406909145064F9720F0109245061092A6
:104FD000440676EDE72E74E0F72E01E02FE130E095
:104FE0004FEF5FEF62E370E08FE090E00E94AE056C
:104FF000EEEBEE2EE4E0FE2E2FE130E04FEF5FEF20
:1050000066E470E08FE090E00E94AE05E090440618
:10501000F090450603E02FE130E04FEF5FEF62E8EC
:1050200070E080E590E00E94F40580916806813090
:1050300009F028C680914406909145064F9720F0CC
:10504000109245061092440656EDE52E54E0F52EDA
:1050500001E02FE130E04FEF5FEF62E370E08FE0BF
:1050600090E00E94AE056EEBE62E64E0F62E2FE196
:1050700030E04FEF5FEF66E470E08FE090E00E9479
:10508000AE05E0904406F0904506F1C5811136C0AA
:1050900080914606909147064F9720F01092470660
:1050A0001092460636EAE32E34E0F32E01E02FE1BB
:1050B00030E04FEF5FEF62E370E08FE090E00E943E
:1050C000AE054EE8E42E44E0F42E2FE130E04FEF41
:1050D0005FEF66E470E08FE090E00E94AE05E09044
:1050E0004606F090470603E02FE130E04FEF5FEF18
:1050F00062E870E080E590E00E94F4058091680627
:10510000813031F48091BB068F5F8093BB0638C03D
:105110008230B1F580914606909147064F9720F076
:10512000109247061092460696EAE92E94E0F92E70
:1051300001E02FE130E04FEF5FEF62E370E08FE0DE
:1051400090E00E94AE052EE8E22E24E0F22E2FE140
:1051500030E04FEF5FEF66E470E08FE090E00E9498
:10516000AE05E0904606F090470603E02FE130E000
:105170004FEF5FEF62E870E080E590E00E94F40599
:10518000809168068430B1F580914606909147067B
:105190004F9720F0109247061092460606EAE02E3E
:1051A00004E0F02E01E02FE130E04FEF5FEF62E32B
:1051B00070E08FE090E00E94AE058EE8E82E84E07B
:1051C000F82E2FE130E04FEF5FEF66E470E08FE004
:1051D00090E00E94AE05E0904606F090470603E09E
:1051E0002FE130E04FEF5FEF62E870E080E590E0A4
:1051F0000E94F405809168068530B1F580914606DD
:10520000909147064F9720F010924706109246065D
:10521000B6EAEB2EB4E0FB2E01E02FE130E04FEFD9
:105220005FEF62E370E08FE090E00E94AE051EE861
:10523000E12E14E0F12E2FE130E04FEF5FEF66E456
:1052400070E08FE090E00E94AE05E0904606F0909E
:10525000470603E02FE130E04FEF5FEF62E870E0D8
:1052600080E590E00E94F40580916806863009F0A0
:10527000F4C580914606909147064F9720F0109212
:10528000470610924606F6EAEF2EF4E0FF2E01E004
:105290002FE130E04FEF5FEF62E370E08FE090E0EE
:1052A0000E94AE05AEE8EA2EA4E0FA2E2FE130E02F
:1052B0004FEF5FEF66E470E08FE090E00E94AE0594
:1052C000E0904606F09047062AC4811145C08091BF
:1052D000480690914906039730F081E090E0909362
:1052E000490680934806E6E7EE2EE4E0FE2E01E054
:1052F0002FE130E04FEF5FEF6CE370E08FE090E084
:105300000E94AE058091480690914906019779F474
:1053100070EAE72E75E0F72E03E02FE130E04FEF63
:105320005FEF62E870E080E590E00E94AE0580915A
:10533000480690914906892B79F46BE9E62E65E0E1
:10534000F62E03E02FE130E04FEF5FEF62E870E010
:1053500080E590E00E94AE0580916806813009F0FA
:1053600045C08091480690914906039730F081E04E
:1053700090E0909349068093480656E7E52E54E066
:10538000F52E01E02FE130E04FEF5FEF6CE370E0CE
:105390008FE090E00E94AE0580914806909149060A
:1053A000019779F440EAE42E45E0F42E03E02FE182
:1053B00030E04FEF5FEF62E870E080E590E00E9440
:1053C000AE058091480690914906892B79F43BE916
:1053D000E32E35E0F32E03E02FE130E04FEF5FEFF7
:1053E00062E870E080E590E00E94AE05809168067A
:1053F000823009F045C08091480690914906039794
:1054000030F081E090E0909349068093480626E7CB
:10541000E22E24E0F22E01E02FE130E04FEF5FEFCB
:105420006CE370E08FE090E00E94AE05809148064A
:1054300090914906019779F490EAE92E95E0F92ECA
:1054400003E02FE130E04FEF5FEF62E870E080E5CE
:1054500090E00E94AE058091480690914906892B04
:1054600079F48BE9E82E85E0F82E03E02FE130E0B7
:105470004FEF5FEF62E870E080E590E00E94AE05DC
:10548000809168069CEF980F923008F4A5C486308E
:1054900009F0E3C48091480690914906039730F0E3
:1054A00081E090E0909349068093480606E7E02E5D
:1054B00004E0F02E01E02FE130E04FEF5FEF6CE30E
:1054C00070E08FE090E00E94AE05809148069091D8
:1054D0004906019779F410EAE12E15E0F12E03E078
:1054E0002FE130E04FEF5FEF62E870E080E590E0A1
:1054F0000E94AE058091480690914906892B09F0DB
:10550000ACC4BBE9EB2EB5E0FB2E03E02FE130E0AD
:105510004FEF5FEF62E870E080E590E00E94AE053B
:105520009CC4811137C080914A0690914B068F35FB
:10553000914020F010924B0610924A06FEE5EF2EA5
:10554000F4E0FF2E01E02FE130E04FEF5FEF62E388
:1055500070E08FE090E00E94AE05A6E4EA2EA4E0A1
:10556000FA2E2FE130E04FEF5FEF66E470E08FE05E
:1055700090E00E94AE05E0904A06F0904B0603E0F2
:105580002FE130E04FEF5FEF62E870E080E590E000
:105590000E94F405809168068130B9F580914A0631
:1055A00090914B068F35914020F010924B0610924F
:1055B0004A067EE5E72E74E0F72E01E02FE130E0A9
:1055C0004FEF5FEF62E370E08FE090E00E94AE0586
:1055D000E6E4EE2EE4E0FE2E2FE130E04FEF5FEF49
:1055E00066E470E08FE090E00E94AE05E0904A062D
:1055F000F0904B0603E02FE130E04FEF5FEF62E801
:1056000070E080E590E00E94F405809168068230A9
:10561000B9F580914A0690914B068F35914020F064
:1056200010924B0610924A065EE5E52E54E0F52EE8
:1056300001E02FE130E04FEF5FEF62E370E08FE0D9
:1056400090E00E94AE0566E4E62E64E0F62E2FE1BF
:1056500030E04FEF5FEF66E470E08FE090E00E9493
:10566000AE05E0904A06F0904B0603E02FE130E0F3
:105670004FEF5FEF62E870E080E590E00E94F40594
:10568000809168069CEF980F923008F4A5C386308D
:1056900009F0E3C380914A0690914B068F35914003
:1056A00020F010924B0610924A063EE5E32E34E0BD
:1056B000F32E01E02FE130E04FEF5FEF62E370E0A7
:1056C0008FE090E00E94AE0546E4E42E44E0F42E24
:1056D0002FE130E04FEF5FEF66E470E08FE090E0A5
:1056E0000E94AE05E0904A06F0904B0618C2811168
:1056F00037C080914C0690914D068636910520F07A
:1057000010924D0610924C069EE2E92E94E0F92E7E
:1057100001E02FE130E04FEF5FEF62E370E08FE0F8
:1057200090E00E94AE0526E1E22E24E0F22E2FE169
:1057300030E04FEF5FEF66E470E08FE090E00E94B2
:10574000AE05E0904C06F0904D0603E02FE130E00E
:105750004FEF5FEF62E870E080E590E00E94F405B3
:10576000809168068130B9F580914C0690914D0684
:105770008636910520F010924D0610924C060EE2EE
:10578000E02E04E0F02E01E02FE130E04FEF5FEF7C
:1057900062E370E08FE090E00E94AE0586E1E82EC3
:1057A00084E0F82E2FE130E04FEF5FEF66E470E029
:1057B0008FE090E00E94AE05E0904C06F0904D0620
:1057C00003E02FE130E04FEF5FEF62E870E080E54B
:1057D00090E00E94F40580916806823031F4809157
:1057E000BB068F5F8093BB0639C08430B9F58091CA
:1057F0004C0690914D068636910520F010924D068C
:1058000010924C06BEE2EB2EB4E0FB2E01E02FE13D
:1058100030E04FEF5FEF62E370E08FE090E00E94D6
:10582000AE0516E1E12E14E0F12E2FE130E04FEF4E
:105830005FEF66E470E08FE090E00E94AE05E090DC
:105840004C06F0904D0603E02FE130E04FEF5FEFA4
:1058500062E870E080E590E00E94F40580916806BF
:105860008530B9F580914C0690914D0686369105AC
:1058700020F010924D0610924C06FEE2EF2EF4E05E
:10588000FF2E01E02FE130E04FEF5FEF62E370E0C9
:105890008FE090E00E94AE05A6E1EA2EA4E0FA2E89
:1058A0002FE130E04FEF5FEF66E470E08FE090E0D3
:1058B0000E94AE05E0904C06F0904D0603E02FE10B
:1058C00030E04FEF5FEF62E870E080E590E00E942B
:1058D000F405809168067DC2811137C080914E0623
:1058E00090914F068636910520F010924F06109247
:1058F0004E067EEFE72E73E0F72E01E02FE130E059
:105900004FEF5FEF62E370E08FE090E00E94AE0542
:10591000E6EEEE2EE3E0FE2E2FE130E04FEF5FEFFC
:1059200066E470E08FE090E00E94AE05E0904E06E5
:10593000F0904F0603E02FE130E04FEF5FEF62E8B9
:1059400070E080E590E00E94F40580916806813067
:1059500031F48091BB068F5F8093BB0639C08230E3
:10596000B9F580914E0690914F068636910520F04C
:1059700010924F0610924E065EEFE52E53E0F52E84
:1059800001E02FE130E04FEF5FEF62E370E08FE086
:1059900090E00E94AE0566EEE62E63E0F62E2FE163
:1059A00030E04FEF5FEF66E470E08FE090E00E9440
:1059B000AE05E0904E06F0904F0603E02FE130E098
:1059C0004FEF5FEF62E870E080E590E00E94F40541
:1059D000809168068430B9F580914E0690914F060B
:1059E0008636910520F010924F0610924E063EEF3B
:1059F000E32E33E0F32E01E02FE130E04FEF5FEFD5
:105A000062E370E08FE090E00E94AE0546EEE42E87
:105A100043E0F42E2FE130E04FEF5FEF66E470E0FB
:105A20008FE090E00E94AE05E0904E06F0904F06A9
:105A300003E02FE130E04FEF5FEF62E870E080E5D8
:105A400090E00E94F405809168068530B9F5809158
:105A50004E0690914F068636910520F010924F0623
:105A600010924E069EEFE92E93E0F92E01E02FE111
:105A700030E04FEF5FEF62E370E08FE090E00E9474
:105A8000AE0526EEE22E23E0F22E2FE130E04FEFBE
:105A90005FEF66E470E08FE090E00E94AE05E0907A
:105AA0004E06F0904F0603E02FE130E04FEF5FEF3E
:105AB00062E870E080E590E00E94F405809168065D
:105AC000863009F0CAC180914E0690914F06863605
:105AD000910520F010924F0610924E061EEFE12E17
:105AE00013E0F12E01E02FE130E04FEF5FEF62E3D2
:105AF00070E08FE090E00E94AE0586EEE82E83E035
:105B0000F82E2FE130E04FEF5FEF66E470E08FE0BA
:105B100090E00E94AE05E0904E06F0904F0603E044
:105B20002FE130E04FEF5FEF62E870E080E590E05A
:105B30000E94F40592C1811129C08091580690916C
:105B400059068D32914020F0109259061092580655
:105B5000B6E6EB2EB3E0FB2E01E02FE130E04FEF95
:105B60005FEF6CE370E08FE090E00E94AE05E090A4
:105B70005806F090590603E02FE130E04FEF5FEF59
:105B800062E870E080E590E00E94F405809168068C
:105B9000813009F077C080915806909159068D3276
:105BA000914020F01092590610925806A6E6EA2E6F
:105BB000A3E0FA2E01E02FE130E04FEF5FEF6CE35E
:105BC00070E08FE090E00E94AE05E0905806F09003
:105BD00059064DC0811129C080915A0690915B06EB
:105BE000893E934020F010925B0610925A06FCEB1F
:105BF000EF2EF3E0FF2E01E02FE130E04FEF5FEFFB
:105C00006CE370E08FE090E00E94AE05E0905A06F1
:105C1000F0905B0603E02FE130E04FEF5FEF62E8CA
:105C200070E080E590E00E94F40580916806813084
:105C300049F580915A0690915B06893E934020F089
:105C400010925B0610925A06ECEBEE2EE3E0FE2E6D
:105C500001E02FE130E04FEF5FEF6CE370E08FE0A9
:105C600090E00E94AE05E0905A06F0905B0603E0DB
:105C70002FE130E04FEF5FEF62E870E080E590E009
:105C80000E94F40580916806823009F4A5C09CEF5B
:105C9000980F923008F09DC09FC0811190C08091F4
:105CA000500690915106039720F0109251061092E1
:105CB000500674EDE72E73E0F72E01E02FE130E09F
:105CC0004FEF5FEF6CE370E08EE190E00E94AE0575
:105CD0008091500690915106019779F460EAE62E82
:105CE00065E0F62E03E02FE130E04FEF5FEF62E872
:105CF00070E080E590E00E94AE05809150069091A2
:105D00005106892B79F45BE9E52E55E0F52E03E089
:105D10002FE130E04FEF5FEF62E870E080E590E068
:105D20000E94AE058091500680932D0648C08111D7
:105D300046C080912D06811108C08DC081113FC0E1
:105D400080912D0681119EC186C0813009F085C0E9
:105D50008091520690915306893E934020F0109214
:105D60005306109252063EE5E32E34E0F32E01E096
:105D70002FE130E04FEF5FEF62E370E08FE090E003
:105D80000E94AE0546EAE42E43E0F42E2FE130E017
:105D90004FEF5FEF66E470E08FE090E00E94AE05A9
:105DA000E0905206F090530603E02FE130E04FEF11
:105DB0005FEF62E870E080E590E00E94F40580917A
:105DC0006806813049F0823039F0843029F085301E
:105DD00019F0863009F041C08091BB068F5F809337
:105DE000BB063BC0882321F09FEF980F923018F438
:105DF0001092BB062BC0843049F580915C069091CF
:105E00005D06893E934020F010925D0610925C067C
:105E10008FE3E82E83E0F82E01E02FE130E04FEF32
:105E20005FEF6CE370E08FE090E00E94AE05E090E1
:105E30005C06F0905D0603E02FE130E04FEF5FEF8E
:105E400062E870E080E590E00E94F40580916806C9
:105E50008550823010F41092BB0680918A06813002
:105E600009F0F3C08093CC061092960680916806E4
:105E7000811128C0E0917006F0917106E830F105BB
:105E800008F5E656FF4F4EE150E00C94C74364E935
:105E900072E014C066E772E011C068E572E00EC0FF
:105EA0006AE372E00BC06CE172E008C06EEF71E073
:105EB00005C060EE71E002C062EC71E080E496E043
:105EC0000E94EF46809168068130E1F4809170066F
:105ED000909171068130910569F038F0029791F444
:105EE0004EE150E068E671E009C04EE150E064EA3E
:105EF00071E004C04EE150E066E871E080E496E0B5
:105F00000E94EF46809168068230E1F4809170062D
:105F1000909171068130910569F038F0029791F403
:105F20004EE150E06EE071E009C04EE150E06AE4FD
:105F300071E004C04EE150E06CE271E080E496E074
:105F40000E94EF46809168068430E1F480917006EB
:105F5000909171068130910569F038F0029791F4C3
:105F60004EE150E064EB70E009C04EE150E060EFBC
:105F700070E004C04EE150E062ED70E080E496E035
:105F80000E94EF46809168068530E1F480917006AA
:105F9000909171068130910569F038F0029791F483
:105FA0004EE150E06AE570E009C04EE150E066E97C
:105FB00070E004C04EE150E068E770E080E496E0F5
:105FC0000E94EF46809168068630E1F48091700669
:105FD000909171068130910569F038F0029791F443
:105FE0004EE150E060E070E009C04EE150E06CE34B
:105FF00070E004C04EE150E06EE170E080E496E0B5
:106000000E94EF468FE190E00E942E068091680684
:10601000811101C075D180916806813009F45CD48A
:1060200080916806823009F45ED5809168068430DC
:1060300009F460D680916806853011F40E94D92455
:1060400080916806863009F453D080918A068111C8
:106050000CC081E08093CC061092960610925E06EA
:106060008FE190E00E942E06EED2C0938A068FE761
:1060700098E321E0815090402040E1F700C000000B
:106080000C94F325813009F0E8CE8091540690916C
:106090005506893E934020F0109255061092540602
:1060A0009FE8E92E93E0F92E01E02FE130E04FEF79
:1060B0005FEF62E370E08FE090E00E94AE052CE7B6
:1060C000E22E23E0F22E2FE130E04FEF5FEF66E4A7
:1060D00070E08FE090E00E94AE05E0905406F090F2
:1060E000550662CECF911F910F91FF90EF900895CA
:1060F000EF92FF920F931F93CF93DF93A895809118
:1061000096068111F6C08FE190E00E942E060E9453
:10611000100F8091BC0690E09093710680937006FA
:1061200085E080938A06C1E0D5E0809196068111D2
:10613000E0C0A8950E94A10F80918A068230A9F440
:1061400080917006909171060196909371068093EC
:1061500070060FE110E02CE330E046EE50E069E617
:1061600070E081E090E00E94B90480918A0683305B
:10617000A9F4809170069091710601979093710631
:10618000809370060FE110E02CE330E046EE50E023
:1061900069E670E081E090E00E94B90480917006A9
:1061A00090917106039720F010927106109270067C
:1061B00080917006909171068130910589F1D0F03F
:1061C000029709F046C081E6E82E85E0F82E02E04D
:1061D0002FE130E04FEF5FEF6DE770E088E290E095
:1061E0000E94AE0582E08093BC064EE150E060E084
:1061F00070E02BC025E7E22E25E0F22E02E02FE131
:1062000030E04FEF5FEF6DE770E088E290E00E94D2
:10621000AE051092BC064EE150E06CE370E015C094
:106220009BE6E92E95E0F92E02E02FE130E04FEFFA
:106230005FEF6DE770E088E290E00E94AE05C093EA
:10624000BC064EE150E06EE170E080E496E00E9412
:10625000D24680918A06811110C0A895C0939606F7
:106260001092770610927606C09385068FE190E033
:106270000E942E06A8950E947B1F80918A0681307D
:1062800061F5A8958093960610927706109276068F
:10629000809385068FE190E00E942E06A8951092CB
:1062A000CC068091BC06813069F038F0823091F4E0
:1062B0004EE150E060E070E009C04EE150E06CE378
:1062C00070E004C04EE150E06EE170E080E496E0E2
:1062D0000E94D246A8950E94DF25D0938A062FEF10
:1062E00080E792E0215080409040E1F700C000003C
:1062F0001CCFDF91CF911F910F91FF90EF900895E8
:10630000AF92BF92CF92DF92EF92FF920F931F93C3
:10631000CF93DF93A89580919606811189C18FE173
:1063200090E00E942E060E94100F8091C00690E01F
:10633000909371068093700685E080938A06E7E06B
:10634000DE2EF6E0CF2ED5E0A4E0BA2EB3E0AB2EE1
:10635000C1E08091960681116BC1A8950E94A10FA2
:1063600080918A068230A9F480917006909171061E
:10637000019690937106809370060FE110E02CE374
:1063800030E046EE50E069E670E081E090E00E9487
:10639000B90480918A068330A9F4809170069091A7
:1063A0007106019790937106809370060FE110E0DB
:1063B0002CE330E046EE50E069E670E081E090E0EA
:1063C0000E94B9048091700690917106089720F0A0
:1063D0001092710610927006E0917006F0917106AD
:1063E000E830F10508F0BEC0EE55FF4F0C94C743EE
:1063F00074E8E72E75E0F72E02E02FE130E04FEF72
:106400005FEF6DE770E082E390E00E94AE051092CE
:10641000C0064EE150E064E972E09AC06FE7E62EF4
:1064200065E0F62E02E02FE130E04FEF5FEF6DE721
:1064300070E082E390E00E94AE05C093C0064EE19A
:1064400050E066E772E084C055E7E52E55E0F52E92
:1064500002E02FE130E04FEF5FEF6DE770E088E2A0
:1064600090E00E94AE0582E08093C0064EE150E0CD
:1064700068E572E06DC04BE6E42E45E0F42E02E0E4
:106480002FE130E04FEF5FEF6DE770E088E290E0E2
:106490000E94AE05A092C0064EE150E06AE372E0B1
:1064A00057C031E6E32E35E0F32E02E02FE130E075
:1064B0004FEF5FEF6DE770E088E290E00E94AE057D
:1064C000B092C00644E150E06CE172E041C027E5C3
:1064D000E22E25E0F22E02E02FE130E04FEF5FEFF9
:1064E0006DE770E088E290E00E94AE05D093C006B0
:1064F0004EE150E06EEF71E02BC09DE4E92E95E097
:10650000F92E02E02FE130E04FEF5FEF6DE770E032
:1065100088E290E00E94AE05C092C0064EE150E0D5
:1065200060EE71E015C083E4E82E85E0F82E02E00D
:106530002FE130E04FEF5FEF6DE770E088E290E031
:106540000E94AE05D092C0064EE150E062EC71E0D0
:1065500080E496E00E94D2468FE59AEE0197F1F72B
:1065600000C0000080918A0681110FC0A895C093D9
:1065700096061092770610927606C09385068FE1F4
:1065800090E00E942E060E947B1F80918A06813037
:1065900009F041C0A8958093960610927706109254
:1065A0007606809385068FE190E00E942E06109279
:1065B000CC06E091C0068E2F90E08830910540F522
:1065C000FC01E655FF4F4EE150E00C94C74364E9EF
:1065D00072E014C066E772E011C068E572E00EC0B8
:1065E0006AE372E00BC06CE172E008C06EEF71E02C
:1065F00005C060EE71E002C062EC71E080E496E0FC
:106600000E94D2468FE59AEE0197F1F700C0000094
:10661000A8950E94DF25D0938A06A8959FEF20E7D2
:1066200082E0915020408040E1F700C0000091CE10
:10663000DF91CF911F910F91FF90EF90DF90CF905E
:10664000BF90AF900895CF93C1E080915E06811115
:1066500041C1E091BB068E2F90E08E30910508F08D
:1066600030C1FC01EE54FF4F0C94C74360914006CB
:106670007091410670933206609331068EE591E089
:106680000E94D84090933206809331069093410641
:10669000809340060DC1609142067091430670934D
:1066A00082066093810682EC91E00E94D84090932C
:1066B0008206809381069093430680934206F8C039
:1066C00060914406709145066093C806772789E17A
:1066D00090E00E94D8408093C80699279093450681
:1066E00080934406E5C0609146067091470660932A
:1066F0006D06772789E190E00E94D84080936D066F
:1067000099279093470680934606D2C08091480609
:10671000809395060E94EF418093950690E09093B8
:10672000490680934806C4C060914A0670914B06A2
:1067300060936C06772788EC90E00E94D8408093A5
:106740006C06992790934B0680934A06B1C06091DE
:106750004C0670914D0660937B06772784E690E0A7
:106760000E94D84080937B06992790934D06809392
:106770004C069EC060914E0670914F0660937A065B
:10678000772784E690E00E94D84080937A06992784
:1067900090934F0680934E068BC06091580670917F
:1067A00059067093B7066093B60688EC90E00E9495
:1067B000D8409093B7068093B6069093590680937D
:1067C000580676C060915A0670915B0670933F063A
:1067D00060933E0684E690E00E94D84090933F0686
:1067E00080933E0690935B0680935A0661C0809129
:1067F000500680932D060E94EF41823018F480935A
:106800002D0602C010922D0680912D0690E09093E7
:106810005106809350064CC080912D06811103C013
:106820001092BB064EC0813009F04BC060915206F9
:10683000709153067093B9066093B8068AEF90E0A2
:106840000E94D8409093B9068093B806909353065F
:10685000809352062DC080912D06882309F3813044
:1068600081F56091540670915506609394067727E0
:1068700086E490E00E94D8408093940699279093F4
:1068800055068093540614C060915C0670915D06B5
:10689000709364066093630684E893E00E94D84096
:1068A000909364068093630690935D0680935C06E4
:1068B0002FE788E391E0215080409040E1F700C04D
:1068C0000000C0935E061092CC060E9400410E9418
:1068D000DF25BBCECF910895EF92FF920F931F93C8
:1068E000CF93DF93A895809196068111F5C08FE133
:1068F00090E00E942E060E94100F80916E0690E09C
:10690000909371068093700685E080938A06C1E0BB
:10691000D5E0809196068111DFC0A8950E94A10F55
:1069200080918A068230A9F4809170069091710658
:10693000019690937106809370060FE110E02CE3AE
:1069400030E046EE50E069E670E081E090E00E94C1
:10695000B90480918A068330A9F4809170069091E1
:106960007106019790937106809370060FE110E015
:106970002CE330E046EE50E069E670E081E090E024
:106980000E94B9048091700690917106039720F0DF
:106990001092710610927006A895809170069091E1
:1069A00071068130910589F1D0F0029709F046C057
:1069B00081E6E82E85E0F82E02E02FE130E04FEF8F
:1069C0005FEF6DE770E088E290E00E94AE0582E044
:1069D00080936E064EE150E068E671E02BC025E73B
:1069E000E22E25E0F22E02E02FE130E04FEF5FEFE4
:1069F0006DE770E088E290E00E94AE0510926E06AE
:106A00004EE150E064EA71E015C09BE6E92E95E0A6
:106A1000F92E02E02FE130E04FEF5FEF6DE770E01D
:106A200088E290E00E94AE05C0936E064EE150E011
:106A300066E871E080E496E00E94D24680918A0682
:106A400081110FC0A895C0939606109277061092F8
:106A50007606C09385068FE190E00E942E060E9484
:106A60007B1F80918A06813059F5A8958093960600
:106A70001092770610927606809385068FE190E05B
:106A80000E942E061092CC0680916E06813069F02D
:106A900038F0823091F44EE150E068E671E009C0D0
:106AA0004EE150E064EA71E004C04EE150E066E877
:106AB00071E080E496E00E94D246A8950E94DF250E
:106AC000D0938A062FEF80E792E0215080409040DB
:106AD000E1F700C000001DCFDF91CF911F910F9112
:106AE000FF90EF900895EF92FF920F931F93CF9333
:106AF000DF93A895809196068111F5C08FE190E013
:106B00000E942E060E94100F8091750690E09093CF
:106B100071068093700685E080938A06C1E0D5E017
:106B2000809196068111DFC0A8950E94A10F8091E7
:106B30008A068230A9F480917006909171060196C0
:106B400090937106809370060FE110E02CE330E023
:106B500046EE50E069E670E081E090E00E94B90402
:106B600080918A068330A9F4809170069091710615
:106B7000019790937106809370060FE110E02CE36B
:106B800030E046EE50E069E670E081E090E00E947F
:106B9000B9048091700690917106039720F01092CD
:106BA0007106109270068091700690917106813086
:106BB000910589F1D0F0029709F046C081E6E82EF0
:106BC00085E0F82E02E02FE130E04FEF5FEF6DE758
:106BD00070E088E290E00E94AE0582E08093750646
:106BE0004EE150E06EE071E02BC025E7E22E25E09B
:106BF000F22E02E02FE130E04FEF5FEF6DE770E043
:106C000088E290E00E94AE05109275064EE150E0D9
:106C10006AE471E015C09BE6E92E95E0F92E02E0EA
:106C20002FE130E04FEF5FEF6DE770E088E290E03A
:106C30000E94AE05C09375064EE150E06CE271E033
:106C400080E496E00E94D24680918A06811110C0AD
:106C5000A895C09396061092770610927606C09378
:106C600085068FE190E00E942E06A8950E947B1F6A
:106C700080918A06813059F5A895809396061092E6
:106C8000770610927606809385068FE190E00E9449
:106C90002E061092CC0680917506813069F038F08E
:106CA000823091F44EE150E06EE071E009C04EE1B7
:106CB00050E06AE471E004C04EE150E06CE271E043
:106CC00080E496E00E94D246A8950E94DF25D093EA
:106CD0008A062FEF80E792E0215080409040E1F754
:106CE00000C000001DCFDF91CF911F910F91FF9049
:106CF000EF900895EF92FF920F931F93CF93DF933E
:106D0000A895809196068111F6C08FE190E00E94CF
:106D10002E060E94100F8091CA0690E09093710693
:106D20008093700685E080938A06C1E0D5E080916B
:106D300096068111E0C0A8950E94A10F80918A0655
:106D40008230A9F48091700690917106019690931B
:106D50007106809370060FE110E02CE330E046EE00
:106D600050E069E670E081E090E00E94B904809113
:106D70008A068330A9F4809170069091710601977C
:106D800090937106809370060FE110E02CE330E0E1
:106D900046EE50E069E670E081E090E00E94B904C0
:106DA0008091700690917106039720F01092710601
:106DB0001092700680917006909171068130910555
:106DC00089F1D0F0029709F046C081E6E82E85E00F
:106DD000F82E02E02FE130E04FEF5FEF6DE770E05B
:106DE00088E290E00E94AE0582E08093CA064EE100
:106DF00050E064EB70E02BC025E7E22E25E0F22E98
:106E000002E02FE130E04FEF5FEF6DE770E088E2E6
:106E100090E00E94AE051092CA064EE150E060EF8D
:106E200070E015C09BE6E92E95E0F92E02E02FE117
:106E300030E04FEF5FEF6DE770E088E290E00E9496
:106E4000AE05C093CA064EE150E062ED70E080E40A
:106E500096E00E94D24680918A06811110C0A895C2
:106E6000C09396061092770610927606C093850618
:106E70008FE190E00E942E06A8950E947B1F8091D2
:106E80008A06813061F5A895809396061092770660
:106E900010927606809385068FE190E00E942E0680
:106EA000A8951092CC068091CA06813069F038F01E
:106EB000823091F44EE150E064EB70E009C04EE1A5
:106EC00050E060EF70E004C04EE150E062ED70E031
:106ED00080E496E00E94D246A8950E94DF25D093D8
:106EE0008A062FEF80E792E0215080409040E1F742
:106EF00000C000001CCFDF91CF911F910F91FF9038
:106F0000EF9008950F931F9380916706811199C0A8
:106F10008091C2069091C3068335910591F581E079
:106F2000809367060E940C150FE110E02CE330E01F
:106F300044E650E06BE470E08EE690E00E94B90415
:106F400024E230E04AE550E064E670E088E090E05A
:106F50000E94B90424E230E04AE550E064E670E0C3
:106F600088E090E00E94B90424E230E04AE550E075
:106F700064E670E08FED90E00E94B9040E947B1FF0
:106F8000A8950E94571E0E94311AA89503E02FE190
:106F900030E04FEF5FEF69E170E085E890E00E943C
:106FA0004F130E94051E0E942F0B809167068130AF
:106FB000A9F5A8950E940C150FE110E02CE330E034
:106FC00044E650E06BE470E08EE690E00E94B90485
:106FD00024E230E04AE550E064E670E088E090E0CA
:106FE0000E94B90424E230E04AE550E064E670E033
:106FF00088E090E00E94B90424E230E04AE550E0E5
:1070000064E670E08FED90E00E94B90480912C0658
:10701000813009F4D0D10E947B1FA8952FEF81EE1B
:1070200094E0215080409040E1F700C000000E94B1
:10703000A5110E942E1E0E9427121F910F910C94E1
:1070400097121F910F9108951F920F920FB60F92F2
:1070500011248F939F938CB190E09093C3068093FB
:10706000C2069F918F910F900FBE0F901F901895A1
:107070001F920F920FB60F9211242F938F939F930D
:1070800080913A0690913B060196883E23E0920754
:1070900028F490933B0680933A0604C010923B0676
:1070A00010923A0680916506811105C01092C506BE
:1070B0001092C4060BC0813049F48091C4069091AF
:1070C000C50601969093C5068093C40680917F06FD
:1070D000811105C010923906109238060BC081301C
:1070E00049F48091380690913906019690933906BB
:1070F0008093380680917806811105C010923D0674
:1071000010923C060BC0813049F480913C0690916E
:107110003D06019690933D0680933C069F918F918A
:107120002F910F900FBE0F901F9018952FEF89E6AB
:1071300098E1215080409040E1F700C000008FEFBF
:107140008ABB81BB80936100C1E0C4BB88EA8FBD6C
:107150008CE08EBD1DBC1CBC17BC16BC8AE78BBD69
:1071600082E18ABD19BC18BC109279001092780097
:1071700080E187BF10BE87E683BF12BE11BE81E8E3
:1071800080938B0085E080938A0010928900109292
:107190008800109281001092800010928700109257
:1071A0008600109285001092840010928300109245
:1071B00082001BB888E98AB986E080939500109216
:1071C00090008FE289B98FE181BD8FE081BD0E947F
:1071D000134281E00E94C5038FE190E00E942E06D9
:1071E000C09367061092680610923B0610923A060A
:1071F00010927D0610923706109266061092C6060F
:1072000010925F0680E590E09093C3068093C206DB
:10721000809164008E7F809364008091650081601E
:107220008093650080916400886080936400809101
:107230006500886080936500C0932C06809164008F
:107240008260809364008091650082608093650015
:107250007894A49AAC9A2FEF85EA9EE02150804062
:107260009040E1F700C00000A895AC9882EB92E056
:107270000E94E246813089F00E94771AA8950E9408
:10728000E41DA89561E083EB92E00E94F846A89582
:1072900061E082EB92E00E94F846A8958091670633
:1072A000813021F4A8950E947B1FA895A8952ADE1D
:1072B000F4CF8091640080618093640080916500C8
:1072C0008061809365008091640088608093640091
:1072D00080916500877F8093650080912206909160
:1072E00023068536910500F58091640084608093C3
:1072F0006400809165008460809365008FEC97E066
:107300000197F1F700C00000A895809165008B7F80
:1073100080936500809122069091230601969093B8
:10732000230680932206D9CF8091650088608093E0
:10733000650008958091640080618093640080916D
:1073400065008F7E809365008091640088608093E3
:10735000640080916500877F80936500809122069C
:10736000909123068536910500F580916400846034
:1073700080936400809165008460809365008FEC49
:1073800097E00197F1F700C00000A8958091650093
:107390008B7F809365008091220690912306019651
:1073A0009093230680932206D9CF80916500886050
:1073B0008093650008958AEB92E00E94E2468093F4
:1073C000CE068091640080618093640080916500A6
:1073D0008061809365008091640088608093640080
:1073E00080916500877F809365008091CE0624E6BA
:1073F000829FC00111242091200630912106281778
:10740000390700F580916400846080936400809166
:1074100065008460809365008FEC97E00197F1F739
:1074200000C00000A895809165008B7F8093650067
:1074300080912006909121060196909321068093D9
:107440002006D3CF809165008860809365001092FC
:10745000260610922106109220060895AC01809114
:10746000260681114AC09091640090619093640057
:10747000909165009F7E9093650090916400986064
:107480009093640090916500977F9093650084E6E7
:10749000849F9001859F300D11248091200690914A
:1074A00021068217930700F5809164008460809321
:1074B0006400809165008460809365008FEC97E0A4
:1074C0000197F1F700C00000A895809165008B7FBF
:1074D00080936500809120069091210601969093FB
:1074E000210680932006D9CF809165008860809323
:1074F0006500109221061092200681E080932606F6
:107500000895682F8AEB92E00C94F8468AEB92E09B
:107510000E94E24690E0A2CF809325060895CF9383
:10752000DF9300D000D0CDB7DEB7809163001C821E
:107530001B821A821982BE016F5F7F4FCE010396B4
:1075400085D78B819C818431954068F489819A81AB
:10755000843A964040F489819A818D32914018F0A6
:1075600082E08093D0068B819C818937954090F092
:107570008B819C81843C994068F489819A81843A0A
:10758000964040F489819A818D32914018F083E0D1
:107590008093D0068B819C8189329A4068F08981E2
:1075A0009A8184379E4040F489819A81813D974039
:1075B00018F081E08093D0068B819C81863F9940B2
:1075C00060F48B819C818134964038F089819A8166
:1075D000813D974010F01092D0068091D0060F9018
:1075E0000F900F900F90DF91CF910895DF92EF925F
:1075F000FF920F931F93CF93DF9385E08093D00684
:10760000DBE485E0D82E8091250681116FC087DFED
:10761000E0902406F12C03E02FE130E040E058EF49
:1076200062E870E080E590E00E94F4058091D00669
:107630008330B1F480912406815080932406109207
:107640002306109222060FE110E02CE330E046EE14
:1076500050E069E670E081E090E00E94B90429DE24
:107660008091D0068230C1F4809124068B34A0F43E
:107670008F5F8093240610922306109222060FE15A
:1076800010E02CE330E046EE50E069E670E081E087
:1076900090E00E94B9044EDE809124068C3410F0F4
:1076A000D09324068091D00681110EC00FE110E026
:1076B0002CE330E046EE50E069E670E081E090E0D7
:1076C0000E94B90410922406C091D006C13059F42A
:1076D0008091240616DF8091240690E06CDE1092E3
:1076E0002406C0932506D092D0068DCFDF91CF918E
:1076F0001F910F91FF90EF90DF900895EF92FF920E
:107700000F931F938AEB92E00E94E2468C3418F4A8
:107710008093CF0613C01092CF0660E08AEB92E010
:107720000E94F8460FE110E028E230E048E550E022
:107730006FEA70E080EE90E00E94B9048091CF067D
:10774000882389F08AEB92E00E94E246E82EF12C31
:1077500002E02FE130E04FEF5FEF6AEA70E080EF88
:1077600090E00E94F4051F910F91FF90EF90089513
:10777000EF92FF920F93E090CF06F12C03E02FE100
:1077800030E04FEF5FEF6AEA70E080EF90E00E9438
:10779000F4050F91FF90EF900895A89521E02093B4
:1077A00065062091C4063091C5062937310578F168
:1077B00020917D0630917E062635310540F5BC01CD
:1077C0002B5F3F4F30937E0620937D061092C506B7
:1077D0001092C40690912806892F90E0880F991F77
:1077E00085549D4F0E940547809128068F5F8093A6
:1077F0002806A49A80E185BBA8952FEF81EE94E03E
:10780000215080409040E1F700C0000015BA089573
:1078100040912706E42FF0E0EE0FFF1FE25FFE4FDE
:107820006081718121E0240F209327066817790772
:1078300020F5E22FF0E0EE0FFF1FE25FFE4F6081C8
:1078400071818617970760F455E0259F90011124F8
:107850002250310930937E0620937D0640932706FF
:1078600020918E0630918F068217930730F48EE1B7
:1078700090E090937E0680937D0680917A0690E05A
:1078800020917D0630917E068217930720F4909315
:107890007E0680937D060895CF93DF9300D000D0BD
:1078A000CDB7DEB78091630080FD6AC01C821B8269
:1078B0001A821982BE016F5F7F4FCE010396C6D533
:1078C0008B819C818531954098F08B819C81883299
:1078D0009A4070F489819A818431954048F480916E
:1078E000CB069091CC0601969093CC068093CB0664
:1078F0008B819C818937954098F08B819C8189325E
:107900009A4070F089819A818431954048F4809141
:10791000CB069091CC0601979093CC068093CB0632
:107920008B819C818531954098F08B819C81883238
:107930009A4070F489819A81853C994048F0809101
:107940007D0690917E06019690937E0680937D063B
:107950008B819C818937954098F08B819C818932FD
:107960009A4070F089819A81853C994048F08091D5
:107970007D0690917E06019790937E0680937D060A
:107980000F900F900F900F90DF91CF910895EF928D
:10799000FF920F931F93CF93DF9300D000D0CDB70A
:1079A000DEB78091100690911106A0911206B09159
:1079B000130689839A83AB83BC8303E02FEF3FEFE9
:1079C0004CED50E068E470E080E090E00E944106F9
:1079D0002FEF3FEF4CED50E06FE770E080E090E07C
:1079E0000E9441062FEF3FEF4CED50E066EB70E058
:1079F00080E090E00E9441062FEF3FEF4CED50E019
:107A00006DEE70E080E090E00E9441062FEF3FEFC6
:107A100045EA50E068E470E080E090E00E94B6063D
:107A20002FEF3FEF45EA50E068E470E087E390E035
:107A30000E94B6062FEF3FEF45EA50E068E470E0A1
:107A40008EE690E00E94B6062FEF3FEF4EE650E044
:107A500068E470E085EA90E00E94B6062FEF3FEF01
:107A600048EA50E068E470E08CED90E00E94B606D1
:107A7000EE24E394F12C2FE130E04FEF5FEF6AE565
:107A800070E08CE090E00E94F40595E0E92EF12C86
:107A90002FE130E04FEF5FEF61E970E08CE090E0C4
:107AA0000E94F40529E0E22EF12C2FE130E04FEFA7
:107AB0005FEF68EC70E08CE090E00E94F40532E04B
:107AC000E32EF12C2FE130E04FEF5FEF6AE570E03D
:107AD00083E490E00E94F40546E0E42EF12C2FE1CF
:107AE00030E04FEF5FEF61E970E083E490E00E94E7
:107AF000F405E12CF12C2FE130E04FEF5FEF68EC63
:107B000070E083E490E00E94F40553E0E52EF12C50
:107B10002FE130E04FEF5FEF6AE570E08AE790E039
:107B20000E94F40567E0E62EF12C2FE130E04FEFE4
:107B30005FEF61E970E08AE790E00E94F40574E08D
:107B4000E72EF12C2FE130E04FEF5FEF6AE570E0B8
:107B500081EB90E00E94F405E8E0EE2EF12C2FE19D
:107B600030E04FEF5FEF61E970E081EB90E00E9461
:107B7000F405E12CF12C2FE130E04FEF5FEF68ECE2
:107B800070E089E890E00E94F4052FE130E04FEFCB
:107B90005FEF68EC70E083EA90E00E94F405F3E0A8
:107BA000EF2E0FEF1FEF2CE330E04AE550E068E4E2
:107BB00070E081EE90E00E942B07CE0101967C01DF
:107BC00002E02FE130E040E058EF64E670E085EF3E
:107BD00090E00E94AE05A3E0EA2E0FEF1FEF20E534
:107BE00030E04AE550E066E970E081EE90E00E9406
:107BF0002B0700EE17E02CED30E04EE051E06EEB8D
:107C000070E085EF90E00E94A80720EA30E04CE2A7
:107C100051E06CED70E08EE091E00E94A8072CED41
:107C200030E04FE051E06EEB70E086EF90E00E94B4
:107C3000A80720EA30E04BE251E06CED70E08DE007
:107C400091E00E94A8072CED30E040E151E06EEB9E
:107C500070E087EF90E00E94A80720EA30E04AE257
:107C600051E06CED70E08CE091E00E94A8072CEDF3
:107C700030E041E151E06EEB70E088EF90E00E946F
:107C8000A80720EA30E04AE251E06CED70E08BE0BA
:107C900091E00E94A807B2E0EB2E0FEF1FEF2CE35C
:107CA00030E040EA50E063E070E080E590E00E9460
:107CB0002B070F900F900F900F90DF91CF911F9196
:107CC0000F91FF90EF900895EF920F931F9383E031
:107CD000E82E0FEF1FEF22E330E040EA50E064E6C9
:107CE00070E084E190E00E942B0720E530E04AE557
:107CF00050E066E970E081EE90E00E942B0700EE14
:107D000017E02CED30E04EE051E06EEB70E085EFD7
:107D100090E00E94A80720EA30E04CE251E06CEDD0
:107D200070E08EE091E00E94A8072CED30E04FE07B
:107D300051E06EEB70E086EF90E00E94A80720EA29
:107D400030E04BE251E06CED70E08DE091E00E949C
:107D5000A8072CED30E040E151E06EEB70E087EFDA
:107D600090E00E94A80720EA30E04AE251E06CED82
:107D700070E08CE091E00E94A8072CED30E041E13A
:107D800051E06EEB70E088EF90E00E94A80720EAD7
:107D900030E04AE251E06CED70E08BE091E00E944F
:107DA000A8071F910F91EF900895EF92FF920F9304
:107DB0001F93CF93DF9300D000D0CDB7DEB77C0107
:107DC0008091630080FD22C11C821B821A8219826D
:107DD000BE016F5F7F4FCE01039638D30FE110E0F5
:107DE0002DE230E042E550E06AE070E08BE990E09F
:107DF0000E94B9048B819C81893B9B4068F08981FA
:107E00009A81883D9E4040F489819A8189349D40C1
:107E100018F089E0809333018B819C818F329940E7
:107E200090F08B819C81803F9A4068F489819A818F
:107E3000883D9E4040F489819A8189349D4018F0A4
:107E400085E0809333018B819C81853A964090F048
:107E50008B819C818C3F984068F489819A81883D10
:107E60009E4040F489819A8189349D4018F081E0D8
:107E7000809333018B819C81853A964090F08B8171
:107E80009C818C3F984068F489819A8188349D4018
:107E900040F489819A818D389A4018F082E080936D
:107EA00033018B819C818F32994090F08B819C8132
:107EB000803F9A4068F489819A8188349D4040F4DB
:107EC00089819A818D389A4018F086E08093330139
:107ED0008B819C81893B9B4060F089819A818834A9
:107EE0009D4038F489819A818D389A4010F0109223
:107EF00033018B819C81893B9B4068F089819A8109
:107F00008E3B9A4040F489819A818F30964018F0D8
:107F10008AE0809333018B819C81853A964090F072
:107F20008B819C818C3F984068F489819A818C3840
:107F30009A4040F489819A81813D974018F083E00E
:107F4000809333018B819C81853A964090F08B81A0
:107F50009C818C3F984068F489819A81803D97404C
:107F600040F489819A818D3D954018F084E080939A
:107F700033018B819C818F32994090F08B819C8161
:107F8000803F9A4068F489819A818C389A4040F405
:107F900089819A81813D974018F087E08093330171
:107FA0008B819C818F32994090F08B819C81803FA6
:107FB0009A4068F489819A81803D974040F4898194
:107FC0009A818D3D954018F088E0809333018B8134
:107FD0009C818D3D954068F08B819C818C3F9840C1
:107FE00040F489819A818C3D954018F48BE0809310
:107FF00033018B819C818F32994040F089819A8135
:108000008C3D954018F48CE08093330180913301CE
:108010008A3088F490912B0691110DC08093D3067D
:1080200090E090932A068093290682E080932B06A5
:108030008EE080933301809133018A30A9F48091DE
:10804000D30634E6839FC001112490932A068093BF
:10805000290622E020932B06E816F90610F08EE0A0
:1080600001C08BE080933301809133018A30C0F4EA
:1080700090912B069230A1F48093D1062091D306E3
:1080800090E04AE0249F800D911D112490932A06D0
:108090008093290683E080932B068EE08093330142
:1080A000209133012A3010F580912B068330F1F4B2
:1080B0002093D2063091D3068091D1064AE0849F66
:1080C000C001112444E6349F800D911D1124820FBC
:1080D000911D90932A068093290621E020932B0678
:1080E000E816F90668F48BE0809333018091330140
:1080F0008B3049F410922A061092290610922B0612
:108100008EE080933301809133018C3019F483E247
:10811000809333010F900F900F900F90DF91CF91CC
:108120001F910F91FF90EF900895EF92FF920F93A0
:10813000E0902906F0902A062AE0E216F10458F4AD
:1081400003E02FE130E04FEF5FEF66E170E088EC95
:1081500090E00E94F405E0902906F0902A06C701FD
:108160000B978935910558F403E02FE130E04FEF8C
:108170005FEF66E170E084EB90E00E94F405E09030
:108180002906F0902A06C701845691098438934045
:1081900058F403E02FE130E04FEF5FEF66E170E06D
:1081A0008BE990E00E94F4050F91FF90EF90089505
:1081B0000F931F93CF93DF93EC018B0180913301D9
:1081C0008E3120F48FE190E00E942E0610932A0653
:1081D00000932906809133018E3128F4D8DBCE013B
:1081E000E4DDA3DFF7CF8FE190E00E942E068091BF
:1081F000290690912A06DF91CF911F910F91089542
:108200008EE0809333010895EF92FF920F931F93B6
:10821000CF93DF93CDB7DEB728970FB6F894DEBFC4
:108220000FBECDBF8091630080FD50C018861F82B5
:108230001E821D82BE016B5F7F4FCE01079606D165
:108240000FE110E02EE230E044E650E062E370E03F
:1082500082E390E00E94B9048F819885853A964028
:1082600090F08F8198858C389A4068F48D819E813A
:1082700084379E4040F48D819E81813F9A4018F062
:1082800081E0809333018F819885853A964088F00C
:108290008F8198858C389A4060F48D819E818C38CE
:1082A0009A4038F48D819E818939984010F010925F
:1082B00033018F8198858F32994040F08D819E8166
:1082C0008C3D954018F48CE080933301809133010C
:1082D000813011F48093320180913201813079F53F
:1082E0008091140690911506A091160689839A83B1
:1082F000AB83CE0101967C0104E02FE130E040EE3B
:1083000057E062E370E086E490E00E94AE0500EE84
:1083100017E02EE230E04DE450E067E670E087E1E0
:1083200090E00E94B9040FE110E02EE230E04DE44D
:1083300050E067E670E086E690E00E94B904809124
:108340003301811102C010923201809132018111FA
:1083500032C08091170690911806A0911906B0912D
:108360001A0689839A83AB83BC8300E018EF2EE260
:1083700030E04DE450E067E670E086E690E00E9471
:10838000B9040FE110E02EE230E04DE450E067E682
:1083900070E087E190E00E94B904CE0101967C0173
:1083A00004E02FE130E040E058EF62E370E087E363
:1083B00090E00E94AE05809133018C3019F483E285
:1083C0008093330128960FB6F894DEBF0FBECDBF61
:1083D000DF91CF911F910F91FF90EF900895CF9370
:1083E000C82F809133018E3120F48FE190E00E94FC
:1083F0002E06C0933201809133018E3120F4A8956E
:1084000063DC02DFF8CF8FE190E00E942E068091BE
:108410003201CF910895C098AB9AAF9A8FB9779BEC
:10842000FECF8FB1089587E087BBC09AAB9AAF9A11
:1084300083E58DB91EB880E8EEDF80E0ECDF80E0F8
:10844000EADF8AE18A95F1F700C00895EF92FF9282
:108450000F931F93CF93DF9300D000D0CDB7DEB73B
:108460007C018B01A895AB9AAF9A1C821B821A8261
:10847000198280EDD0DF80E0CEDF8FB190E09C8369
:108480008B838B819C81982F88279C838B8380E0B2
:10849000C2DF2FB18B819C81822B9C838B838B814C
:1084A0009C8133E0969587953A95E1F79C838B8381
:1084B00087EC90E00197F1F700C0000080E9ABDFA6
:1084C00080E0A9DF8FB190E09A83898389819A81C6
:1084D000982F88279A83898380E09DDF2FB1898137
:1084E0009A81822B9A83898389819A8153E0969518
:1084F00087955A95E1F79A8389832B813C8182ED98
:108500009FE0821B930BF7019183808389819A817D
:10851000F801918380830F900F900F900F90DF915F
:10852000CF911F910F91FF90EF90089570D088F038
:108530009F5790F0B92F9927B751A0F0D1F0660F4F
:10854000771F881F991F1AF0BA95C9F712C0B1306A
:1085500081F077D0B1E0089574C0672F782F882715
:10856000B85F39F0B93FCCF3869577956795B395A9
:10857000D9F73EF490958095709561957F4F8F4F18
:108580009F4F0895E89409C097FB3EF4909580951D
:10859000709561957F4F8F4F9F4F9923A9F0F92FC9
:1085A00096E9BB279395F695879577956795B79547
:1085B000F111F8CFFAF4BB0F11F460FF1BC06F5F2D
:1085C0007F4F8F4F9F4F16C0882311F096E911C03F
:1085D000772321F09EE8872F762F05C0662371F060
:1085E00096E8862F70E060E02AF09A95660F771F74
:1085F000881FDAF7880F9695879597F9089557FDA4
:108600009058440F551F59F05F3F71F04795880F00
:1086100097FB991F61F09F3F79F087950895121697
:1086200013061406551FF2CF4695F1DF08C0161643
:1086300017061806991FF1CF8695710561050894F4
:108640000895E894BB2766277727CB0197F908950B
:108650000BD078C069D028F06ED018F0952309F0BF
:108660005AC05FC01124EECFCADFA0F3959FD1F3AB
:10867000950F50E0551F629FF001729FBB27F00DD0
:10868000B11D639FAA27F00DB11DAA1F649F662725
:10869000B00DA11D661F829F2227B00DA11D621F74
:1086A000739FB00DA11D621F839FA00D611D221F2E
:1086B000749F3327A00D611D231F849F600D211D12
:1086C000822F762F6A2F11249F5750408AF0E1F0B5
:1086D00088234AF0EE0FFF1FBB1F661F771F881FFE
:1086E00091505040A9F79E3F510570F014C0AACF99
:1086F0005F3FECF3983EDCF3869577956795B795E9
:10870000F795E7959F5FC1F7FE2B880F911D969512
:10871000879597F9089597F99F6780E870E060E082
:1087200008959FEF80EC089500240A94161617060A
:1087300018060906089500240A9412161306140652
:1087400005060895092E0394000C11F4882352F0B5
:10875000BB0F40F4BF2B11F460FF04C06F5F7F4F6D
:108760008F4F9F4F0895AA1BBB1B51E107C0AA1F43
:10877000BB1FA617B70710F0A61BB70B881F991FC2
:108780005A95A9F780959095BC01CD010895EE0FFB
:10879000FF1F0024001C0BBE0790F691E02D0994EA
:1087A000A29FB001B39FC001A39F700D811D112432
:1087B000911DB29F700D811D1124911D0895BB273D
:1087C0004A3031F4992322F4BDE2909581959F4F70
:1087D00001C0BB27FB015527AA27880F991FAA1F95
:1087E000A41710F0A41B83955051B9F7A05DAA33CC
:1087F00008F0A95DA193009779F7B111B193119297
:10880000CB0126C2CF93DF93CDB7DEB7AE014B5F6E
:108810005F4FFA0161917191AF018091D6069091FD
:10882000D70603D0DF91CF9108952F923F924F92B8
:108830005F926F927F928F929F92AF92BF92CF92F0
:10884000DF92EF92FF920F931F93CF93DF93CDB7F9
:10885000DEB72B970FB6F894DEBF0FBECDBF6C010D
:108860007B018A01FC0117821682838181FFBFC1CF
:10887000CE0101963C01F6019381F70193FD8591AC
:1088800093FF81917F01882309F4ADC1853239F4CA
:1088900093FD859193FF81917F01853221F4B6018B
:1088A00090E0E6D1E8CF912C212C312CFFE1F3159B
:1088B000D8F08B3279F038F4803279F08332A1F439
:1088C000232D20611DC08D3261F0803369F4232D8A
:1088D000216016C0832D8260382EE32DE4603E2E89
:1088E0002AC0F32DF8601DC037FC2DC020ED280FE5
:1088F0002A3040F08E32B9F436FC75C1232D206445
:10890000322E19C036FE06C08AE0989E200D112432
:10891000922E11C0EAE02E9E200D1124222EF32D5E
:10892000F0623F2E08C08C3621F4832D8068382EEB
:1089300002C0883641F4F70193FD859193FF819140
:108940007F018111B3CF982F9F7D9554933028F4E8
:108950000C5F1F4F9FE399830DC0833631F083373F
:1089600071F0833509F055C020C0F80180818983FA
:108970000E5F1F4F88248394912C530112C028014D
:10898000F2E04F0E511CF801A080B18036FE03C00A
:10899000692D70E002C06FEF7FEFC5014ED14C0131
:1089A0008201F32DFF773F2E15C0280122E0420EF1
:1089B000511CF801A080B18036FE03C0692D70E023
:1089C00002C06FEF7FEFC5012DD14C01F32DF06890
:1089D0003F2E820133FC19C0822D90E08816990643
:1089E000A0F4B60180E290E043D12A94F5CFF501DE
:1089F00037FC859137FE81915F01B60190E038D157
:108A000021102A9421E0821A91088114910479F7A7
:108A1000E1C0843611F0893639F5F80137FE07C018
:108A200060817181828193810C5F1F4F08C06081DA
:108A30007181072E000C880B990B0E5F1F4FF32DD1
:108A4000FF763F2E97FF09C09095809570956195B0
:108A50007F4F8F4F9F4FF0683F2E2AE030E0A301F9
:108A600043D1882E861844C0853731F4232D2F7EBC
:108A7000B22E2AE030E025C0932D997FB92E8F3693
:108A8000C1F018F4883579F0AEC0803719F0883716
:108A900021F0A9C0E92FE061BE2EB4FE0DC0FB2D70
:108AA000F460BF2E09C034FE0AC0292F2660B22E02
:108AB00006C028E030E005C020E130E002C020E13F
:108AC00032E0F801B7FE07C0608171818281938135
:108AD0000C5F1F4F06C06081718180E090E00E5FE7
:108AE0001F4FA30101D1882E8618FB2DFF773F2E43
:108AF00036FE0DC0232D2E7FA22E891458F434FE8D
:108B00000BC032FC09C0832D8E7EA82E05C0B82C68
:108B1000A32C03C0B82C01C0B92CA4FE0FC0FE01C9
:108B2000E80DF11D8081803321F49A2D997EA92EC4
:108B300009C0A2FE06C0B394B39404C08A2D8678FF
:108B400009F0B394A3FC10C0A0FE06C0B21480F4D8
:108B5000280C922C9B180DC0B21458F4B60180E278
:108B600090E086D0B394F8CFB21418F42B1802C05A
:108B7000982C212CA4FE0FC0B60180E390E078D0A1
:108B8000A2FE16C0A1FC03C088E790E002C088E501
:108B900090E0B6010CC08A2D867851F0A1FE02C08B
:108BA0008BE201C080E2A7FC8DE2B60190E060D0CC
:108BB000891430F4B60180E390E05AD09A94F8CF4B
:108BC0008A94F301E80DF11D8081B60190E050D048
:108BD0008110F6CF222009F44ECEB60180E290E05B
:108BE00047D02A94F7CFF6018681978102C08FEF94
:108BF0009FEF2B960FB6F894DEBF0FBECDBFDF916F
:108C0000CF911F910F91FF90EF90DF90CF90BF9089
:108C1000AF909F908F907F906F905F904F903F901C
:108C20002F900895FC010590615070400110D8F715
:108C3000809590958E0F9F1F0895FC0161507040A4
:108C400001900110D8F7809590958E0F9F1F089581
:108C5000DC01FC01672F71917723E1F7329704C0A3
:108C60007C916D9370836291AE17BF07C8F308952E
:108C70000F931F93CF93DF93FB01238121FD03C04B
:108C80008FEF9FEF2CC022FF16C0468157812481B1
:108C900035814217530744F4A081B1819D012F5FB4
:108CA0003F4F318320838C93268137812F5F3F4F45
:108CB0003783268314C08B01EC01FB010084F1850E
:108CC000E02D0995892BE1F6D80116968D919C919E
:108CD0001797019617969C938E931697CE01DF9166
:108CE000CF911F910F910895FA01AA27283051F1D1
:108CF000203181F1E8946F936E7F6E5F7F4F8F4FCD
:108D00009F4FAF4FB1E03ED0B4E03CD0670F781F2B
:108D1000891F9A1FA11D680F791F8A1F911DA11D10
:108D20006A0F711D811D911DA11D20D009F4689449
:108D30003F912AE0269F11243019305D3193DEF6F1
:108D4000CF010895462F4770405D4193B3E00FD0A7
:108D5000C9F7F6CF462F4F70405D4A3318F0495D92
:108D600031FD4052419302D0A9F7EACFB4E0A69575
:108D70009795879577956795BA95C9F70097610597
:108D8000710508959B01AC010A2E069457954795ED
:108D900037952795BA95C9F7620F731F841F951FE2
:108DA000A01D0895DC01CB01FC01E199FECF06C0B6
:108DB000FFBBEEBBE09A31960DB20D924150504090
:108DC000B8F70895E199FECF9FBB8EBBE09A992733
:108DD0008DB30895A8E1B0E042E050E0E5CFDC01BA
:108DE000CB0102C02D9105D041505040D8F70895D5
:108DF000262FE199FECF9FBB8EBB2DBB0FB6F894FB
:108E0000E29AE19A0FBE01960895F2DF272FF1CF83
:048E1000F894FFCF04
:108E14000000000200000000160900000000140019
:108E240048005D0078009600B600D500F3001001FC
:108E34002C01490163017C019401AC01C101D501FC
:108E4400E801010E2020D1F2E0EDF6E8FF00C2E5D2
:108E5400F0F5EDE8E900CDE8E6EDE8E900D0F3F758
:108E6400EDEEE900D0E5E1EEEBEBE8EDE32000D137
:108E7400F3F8EAE000ECE8EAF0EEF1F5E5EC00EFF7
:108E8400EBE0F20020D1F2E5EAEBEE00CAE0EBE819
:108E9400E1F0EEE2EAE000EDE8E7E000CCEEF9ED27
:108EA400EEF1F2FC00E2E5F0F5E000C2E5F0F5EDEC
:108EB400E8E920EDE0E3F02E00CDE8E6EDE8E92076
:108EC400EDE0E3F02E20002020D0F3F7EDEEE920D2
:108ED400202000C4EEEF2E20EDE0F1F2F0EEE9EAFE
:108EE400E800CAE0EBE8E1F0EEE2EAE02000EDE8B9
:108EF400E7E02000C2DBD5CEC40057543D202575E1
:108F04000A47530047533D2025750A534E00534EDC
:108F14003D2025750A454E4400574B3D2025750AD2
:108F2400565000503D332E360A5200524C3D2025F7
:108F3400750A68004F3D73740A5300473D73740A01
:108F4400530053523D53746174696F6E200A575035
:108F54000057503D536E36332F506233370A5754FF
:108F64000057503D536E41670A57540057503D50C7
:108F7400726F66696C65300A57540057503D5072E1
:108F84006F66696C65310A57540057503D50726FD3
:108F940066696C65320A57540057503D50726F66CB
:108FA400696C65330A57540057503D50726F6669B7
:108FB4006C65340A57540057503D50726F66696CA3
:108FC40065350A57540053523D55506865617465C0
:108FD40072200A57500053523D507265686561749F
:108FE4006572200A57500053523D4D616E75616C95
:108FF400200A57500053523D5265626F6C6C696E83
:1090040067200A57500053523D4368697068656190
:1090140074696E67200A57500053523D50434268AA
:10902400656174696E67200A57500053523D50437E
:10903400200A575000C2FBE1E5F0E8F2E520E2FB2C
:10904400F1EEF2F3004D6963726F56322E30002058
:109054002020C2F0E5ECFF20F0E5E1EEEBEBE8EDDB
:10906400E3E02020202000C2FBE1E5F0E8F2E52067
:10907400F0E5E6E8EC00D2E5ECEFE5F0E0F2F3F041
:10908400E020EFEEEBEEF7EAE8202000EDE8E7E081
:1090940020EFF0E820E4EEEDE0E3F0E5E2E500D2D5
:1090A400E5ECEFE5F0E0F2F3F0E020F3E2E5EBE8E5
:1090B400F7E5EDE8FF00202020202020E4EEEDE09D
:1090C400E3F0E5E2E020202020202000C4EBE8F2D9
:1090D400E5EBFCEDEEF1F2FC20E2EFE8F2FBE2E07E
:1090E400EDE8FF00D4F3EDEAF6E8FF20E4EEEDEE60
:1090F400E3F0E5E2E000EDE8E6EDE5E3EE20EDE0A7
:10910400E3F0E5E2E0F2E5EBFF2020202000CCE0F4
:10911400EAF1E8ECE0EBFCEDE0FF20ECEEF9EDEE3B
:10912400F1F2FC202000E2E5F0F5EDE5E3EE20EDC0
:10913400E0E3F0E5E2E0F2E5EBFF20202000CCE004
:10914400EAF1E8ECE0EBFCEDE0FF20ECEEF9EDEE0B
:10915400F1F2FC202000E2E5F0F5EDE5E3EE20ED90
:10916400E0E3F0E5E2E0F2E5EBFF20202000D2E5C9
:10917400ECEFE5F0E0F2F3F0E020E2EAEBFEF7E5F5
:10918400EDE8FF202000CAEEEDF2F0EEEBFC20EF5C
:10919400EE20E2E5F0F5F320202020202000EDE889
:1091A400E6EDE5E3EE20EDE0E3F0E5E2E0F2E5EB09
:1091B400FF2020202000CAEEFDF4F4E8F6E8E5EDF7
:1091C400F220EFF0EEF4E8EBFF2020202000E2E5AF
:1091D400F0F5EDE5E3EE20EDE0E3F0E5E2E0F2E5C5
:1091E400EBFF20202000CAEEFDF4F4E8F6E8E5EDFC
:1091F400F220EFF0EEF4E8EBFF2020202000EDE079
:10920400E3F0E5E2E0F2E5EBFF202000D2E5ECEF4D
:10921400E5F0E0F2F3F0E020EDE8E6EDE5E3EE2042
:1092240020202000EFE0E9EAE82000D2E5ECEFE5B9
:10923400F0E0F2F3F0E020ECE5F1F2E02020202071
:109244002000C2FBE1E5F0E8F2E520EFF0EEF4E8FF
:10925400EBFC00CFF0EEF4E8EBFC203500CFF0EEB1
:10926400F4E8EBFC203400CFF0EEF4E8EBFC203320
:1092740000CFF0EEF4E8EBFC203200CFF0EEF4E89F
:10928400EBFC203100CFF0EEF4E8EBFC203000538F
:109294006E416700536E506200CFF0E8EDFFF2EECE
:1092A400202000C2DBC1D0C0D2DC00C2DBCACB00AC
:1092B400C2CACB00CDE0F1F2F0EEE8F2FC00C7E266
:1092C400F3EAEEE2FBE520F1E8E3EDE0EBFB00CFAF
:1092D400F0E5E4F3F1F2E0EDEEE2EAE800D3ECEEDF
:1092E400EBF7E0EDE8FF00C2F0E5ECFF20EFE0E98A
:1092F400EAE80020C4E0F2F7E8EA20EDE8E62E20F0
:10930400EDE0E3F0E5E2E0F2E5EBFF0020C4E0F29B
:10931400F7E8EA20ECE5F1F2E020EFE0E9EAE80022
:0C93240044656C004F4E004F46460000B0
:00000001FF
